:020000040800F2
:104000000000012065960008098900080B89000856
:104010000D8900080F8900081189000800000000C0
:1040200000000000000000000000000013890008EC
:104030001589000800000000178900081989000888
:10404000AD960008AD960008AD960008AD96000844
:10405000AD960008AD960008AD960008AD96000834
:10406000AD960008AD960008AD9600081D890008C1
:10407000AD960008AD96000829890008358900082A
:10408000AD960008AD960008AD960008AD96000804
:10409000AD960008AD960008AD960008AD960008F4
:1040A000AD960008AD960008AD960008AD960008E4
:1040B000AD960008AD960008AD960008AD960008D4
:1040C000AD960008AD960008AD960008AD960008C4
:1040D000AD96000841890008AD960008AD9600082D
:1040E000AD960008AD960008AD960008AD960008A4
:1040F000AD960008AD960008AD960008AD96000894
:10410000AD960008AD960008AD960008AD96000883
:10411000AD960008AD9600084D890008AD960008E0
:10412000AD960008AD960008AD960008AD96000863
:10413000000000000000000000000000000000007F
:10414000000000000000000000000000000000006F
:10415000000000000000000000000000000000005F
:10416000000000000000000000000000000000004F
:10417000000000000000000000000000000000003F
:10418000000000000000000000000000000000002F
:10419000000000000000000000000000000000001F
:1041A000000000000000000000000000000000000F
:1041B00000000000000000000000000000000000FF
:1041C00000000000000000000000000000000000EF
:1041D00000000000000000000000000000000000DF
:0441E0005FF8E0F1B3
:1041E80010B5054C237833B9044B13B10448AFF329
:1041F80000800123237010BD20040020000000006F
:10420800E4BF000808B5034B1BB103490348AFF3EB
:10421800008008BD0000000024040020E4BF00085E
:10422800034613F8012B002AFBD1181A01387047EE
:10423800D0400B1CD1409C46203AD34018435242F0
:10424800634693401843704781F0004102E000BF85
:1042580083F0004330B54FEA41044FEA430594EA3E
:10426800050F08BF90EA020F1FBF54EA000C55EA79
:10427800020C7FEA645C7FEA655C00F0E2804FEA4A
:104288005454D4EB5555B8BF6D420CDD2C4480EA2C
:10429800020281EA030382EA000083EA010180EA5C
:1042A800020281EA0303362D88BF30BD11F0004FAA
:1042B8004FEA01314FF4801C4CEA113102D04042E0
:1042C80061EB410113F0004F4FEA03334CEA13331B
:1042D80002D0524263EB430394EA050F00F0A78033
:1042E800A4F10104D5F1200E0DDB02FA0EFC22FA2E
:1042F80005F2801841F1000103FA0EF2801843FA22
:1043080005F359410EE0A5F120050EF1200E012A12
:1043180003FA0EFC28BF4CF0020C43FA05F3C01850
:1043280051EBE37101F0004507D54FF0000EDCF1C9
:10433800000C7EEB00006EEB0101B1F5801F1BD372
:10434800B1F5001F0CD349085FEA30004FEA3C0C76
:1043580004F101044FEA445212F5800F80F09A806C
:10436800BCF1004F08BF5FEA500C50F1000041EB70
:10437800045141EA050130BD5FEA4C0C404141EB74
:10438800010111F4801FA4F10104E9D191F0000F9B
:1043980004BF01460020B1FA81F308BF2033A3F11E
:1043A8000B03B3F120020CDA0C3208DD02F1140C15
:1043B800C2F10C0201FA0CF021FA02F10CE002F150
:1043C8001402D8BFC2F1200C01FA02F120FA0CFC49
:1043D800DCBF41EA0C019040E41AA2BF01EB045192
:1043E800294330BD6FEA04041F3C1CDA0C340EDC90
:1043F80004F11404C4F1200220FA04F001FA02F3D3
:1044080040EA030021FA04F345EA030130BDC4F190
:104418000C04C4F1200220FA02F001FA04F340EA85
:104428000300294630BD21FA04F0294630BD94F036
:10443800000F83F4801306BF81F480110134013D1D
:104448004EE77FEA645C18BF7FEA655C29D094EA8E
:10445800050F08BF90EA020F05D054EA000C04BF0C
:104468001946104630BD91EA030F1EBF00210020F7
:1044780030BD5FEA545C05D14000494128BF41F096
:10448800004130BD14F580043CBF01F5801130BDFA
:1044980001F0004545F0FE4141F470014FF0000085
:1044A80030BD7FEA645C1ABF194610467FEA655C36
:1044B8001CBF0B46024650EA013406BF52EA0335D8
:1044C80091EA030F41F4002130BD00BF90F0000FC6
:1044D80004BF0021704730B54FF4806404F1320402
:1044E8004FF000054FF0000150E700BF90F0000FBB
:1044F80004BF0021704730B54FF4806404F13204E2
:1045080010F0004548BF40424FF000013EE700BFB1
:1045180042004FEAE2014FEA31014FEA02701FBF41
:1045280012F07F4393F07F4F81F06051704792F013
:10453800000F14BF93F07F4F704730B54FF460748D
:1045480001F0004521F0004120E700BF50EA0102D8
:1045580008BF704730B54FF000050AE050EA010285
:1045680008BF704730B511F0004502D5404261EBF5
:1045780041014FF4806404F132045FEA915C3FF436
:10458800DCAE4FF003025FEADC0C18BF03325FEACF
:10459800DC0C18BF033202EBDC02C2F1200300FA84
:1045A80003FC20FA02F001FA03FE40EA0E0021FAA9
:1045B80002F11444C1E600BF70B54FF0FF0C4CF493
:1045C800E06C1CEA11541DBF1CEA135594EA0C0F49
:1045D80095EA0C0F00F0DEF82C4481EA030621EA84
:1045E8004C5123EA4C5350EA013518BF52EA0335BF
:1045F80041F4801143F4801338D0A0FB02CE4FF071
:104608000005E1FB02E506F00042E0FB03E54FF0A0
:104618000006E1FB03569CF0000F18BF4EF0010E98
:10462800A4F1FF04B6F5007F64F5407404D25FEA94
:104638004E0E6D4146EB060642EAC62141EA555147
:104648004FEAC52040EA5E504FEACE2EB4F1FD0C89
:1046580088BFBCF5E06F1ED8BEF1004F08BF5FEA07
:10466800500E50F1000041EB045170BD06F00046B9
:1046780046EA010140EA020081EA0301B4EB5C0466
:10468800C2BFD4EB0C0541EA045170BD41F480115E
:104698004FF0000E013C00F3AB8014F1360FDEBF83
:1046A800002001F0004170BDC4F10004203C35DA5F
:1046B8000C341BDC04F11404C4F1200500FA05F3E2
:1046C80020FA04F001FA05F240EA020001F0004283
:1046D80021F0004110EBD37021FA04F642EB0601F9
:1046E8005EEA430E08BF20EAD37070BDC4F10C0423
:1046F800C4F1200500FA04F320FA05F001FA04F2E7
:1047080040EA020001F0004110EBD37041F10001D2
:104718005EEA430E08BF20EAD37070BDC4F12005DD
:1047280000FA05F24EEA020E20FA04F301FA05F245
:1047380043EA020321FA04F001F0004121FA04F2ED
:1047480020EA020000EBD3705EEA430E08BF20EABD
:10475800D37070BD94F0000F0FD101F000464000F7
:1047680041EB010111F4801F08BF013CF7D041EA79
:10477800060195F0000F18BF704703F0004652007D
:1047880043EB030313F4801F08BF013DF7D043EA4E
:104798000603704794EA0C0F0CEA135518BF95EA04
:1047A8000C0F0CD050EA410618BF52EA4306D1D18B
:1047B80081EA030101F000414FF0000070BD50EAAA
:1047C800410606BF1046194652EA430619D094EA34
:1047D8000C0F02D150EA013613D195EA0C0F05D11E
:1047E80052EA03361CBF104619460AD181EA030172
:1047F80001F0004141F0FE4141F470014FF000002A
:1048080070BD41F0FE4141F4780170BD70B54FF0C4
:10481800FF0C4CF4E06C1CEA11541DBF1CEA135544
:1048280094EA0C0F95EA0C0F00F0A7F8A4EB050426
:1048380081EA030E52EA03354FEA013100F088801D
:104848004FEA03334FF0805545EA131343EA1263E6
:104858004FEA022245EA111545EA10654FEA00269B
:104868000EF000419D4208BF964244F1FD0404F554
:10487800407402D25B084FEA3202B61A65EB0305B0
:104888005B084FEA32024FF480104FF4002CB6EB6D
:10489800020E75EB030E22BFB61A754640EA0C00ED
:1048A8005B084FEA3202B6EB020E75EB030E22BF2D
:1048B800B61A754640EA5C005B084FEA3202B6EB6E
:1048C800020E75EB030E22BFB61A754640EA9C002D
:1048D8005B084FEA3202B6EB020E75EB030E22BFFD
:1048E800B61A754640EADC0055EA060E18D04FEABB
:1048F800051545EA16754FEA06164FEAC30343EA5B
:1049080052734FEAC2025FEA1C1CC0D111F4801F27
:104918000BD141EA00014FF000004FF0004CB6E720
:1049280011F4801F04BF01430020B4F1FD0C88BFBF
:10493800BCF5E06F3FF6AFAEB5EB030C04BFB6EBCA
:10494800020C5FEA500C50F1000041EB045170BDBD
:104958000EF0004E4EEA113114EB5C04C2BFD4EBEA
:104968000C0541EA045170BD41F480114FF0000E6E
:10497800013C90E645EA060E8DE60CEA135594EAEA
:104988000C0F08BF95EA0C0F3FF43BAF94EA0C0FED
:104998000AD150EA01347FF434AF95EA0C0F7FF462
:1049A80025AF104619462CE795EA0C0F06D152EAB6
:1049B80003353FF4FDAE1046194622E750EA41069A
:1049C80018BF52EA43067FF4C5AE50EA41047FF4AB
:1049D8000DAF52EA43057FF4EBAE12E74FF0FF3C10
:1049E80006E000BF4FF0010C02E000BF4FF0010CE1
:1049F8004DF804CD4FEA410C7FEA6C5C4FEA430C5A
:104A080018BF7FEA6C5C1BD001B050EA410C0CBFA8
:104A180052EA430C91EA030F02BF90EA020F00200A
:104A2800704710F1000F91EA030F58BF994208BF71
:104A380090422CBFD8176FEAE37040F0010070472E
:104A48004FEA410C7FEA6C5C02D150EA013C07D185
:104A58004FEA430C7FEA6C5CD6D152EA033CD3D0D0
:104A68005DF8040B704700BF8446104662468C46CA
:104A78001946634600E000BF01B5FFF7B7FF0028FD
:104A880048BF10F1000F01BD4DF808EDFFF7F4FF26
:104A98000CBF012000205DF808FB00BF4DF808EDB1
:104AA800FFF7EAFF34BF012000205DF808FB00BFD4
:104AB8004DF808EDFFF7E0FF94BF012000205DF8F6
:104AC80008FB00BF4DF808EDFFF7CEFF94BF0120AB
:104AD80000205DF808FB00BF4DF808EDFFF7C4FFA4
:104AE80034BF012000205DF808FB00BF4FEA410CED
:104AF8007FEA6C5C02D150EA013C0AD14FEA430CD0
:104B08007FEA6C5C02D152EA033C02D14FF000000C
:104B180070474FF0010070474FEA410212F500124A
:104B280015D211D56FF47873B3EB625212D94FEAEC
:104B3800C12343F0004343EA505311F0004F23FAD6
:104B480002F018BF404270474FF00000704750EA2B
:104B5800013005D111F0004008BF6FF000407047E8
:104B68004FF00000704700BF4A0011D212F5001242
:104B780011D20DD56FF47873B3EB62520ED44FEAAD
:104B8800C12343F0004343EA505323FA02F070472D
:104B98004FF00000704750EA013002D14FF0FF306B
:104BA80070474FF0000070474FEA4102B2F1E0430E
:104BB80024BFB3F5001CDCF1FE5C0DD901F0004CFC
:104BC8004FEAC0024CEA5070B2F1004F40EB83004C
:104BD80008BF20F00100704711F0804F21D113F178
:104BE8003872BCBF01F00040704741F480114FEAB1
:104BF8005252C2F11802C2F1200C10FA0CF320FA3A
:104C080002F018BF40F001004FEAC1234FEAD32356
:104C180003FA0CFC40EA0C0023FA02F34FEA4303C0
:104C2800CCE77FEA625307D150EA01331EBF4FF049
:104C3800FE4040F44000704701F0004040F0FE4064
:104C480040F40000704700BF80F0004002E000BF61
:104C580081F0004142001FBF5FEA410392EA030F5F
:104C68007FEA226C7FEA236C6AD04FEA1262D2EBA9
:104C78001363C1BFD218414048404140B8BF5B42AE
:104C8800192B88BF704710F0004F40F4000020F047
:104C98007F4018BF404211F0004F41F4000121F05D
:104CA8007F4118BF494292EA030F3FD0A2F10102A7
:104CB80041FA03FC10EB0C00C3F1200301FA03F1E5
:104CC80000F0004302D5494260EB4000B0F5000F08
:104CD80013D3B0F1807F06D340084FEA310102F1C7
:104CE8000102FE2A51D2B1F1004F40EBC25008BF79
:104CF80020F0010040EA03007047490040EB000043
:104D080010F4000FA2F10102EDD1B0FA80FCACF171
:104D1800080CB2EB0C0200FA0CF0AABF00EBC25070
:104D280052421843BCBFD0401843704792F0000F5E
:104D380081F4000106BF80F400000132013BB5E7B1
:104D48004FEA41037FEA226C18BF7FEA236C21D027
:104D580092EA030F04D092F0000F08BF084670478C
:104D680090EA010F1CBF0020704712F07F4F04D15A
:104D7800400028BF40F00040704712F100723CBF6D
:104D880000F50000704700F0004343F0FE4040F497
:104D9800000070477FEA226216BF08467FEA236355
:104DA8000146420206BF5FEA412390EA010F40F440
:104DB800800070474FF0000304E000BF10F000438C
:104DC80048BF40425FEA000C08BF704743F0964373
:104DD80001464FF000001CE050EA010208BF70478E
:104DE8004FF000030AE000BF50EA010208BF704715
:104DF80011F0004302D5404261EB41015FEA010C2A
:104E080002BF84460146002043F0B64308BFA3F121
:104E18008053A3F50003BCFA8CF2083AA3EBC25303
:104E280010DB01FA02FC634400FA02FCC2F1200222
:104E3800BCF1004F20FA02F243EB020008BF20F059
:104E48000100704702F1200201FA02FCC2F12002BF
:104E580050EA4C0021FA02F243EB020008BF20EAB4
:104E6800DC7070474FF0FF0C1CEAD0521EBF1CEAE2
:104E7800D15392EA0C0F93EA0C0F6FD01A4480EAD0
:104E8800010C400218BF5FEA41211ED04FF00063B9
:104E980043EA501043EA5111A0FB01310CF00040E5
:104EA800B1F5000F3EBF490041EAD3715B0040EA0B
:104EB800010062F17F02FD2A1DD8B3F1004F40EBDB
:104EC800C25008BF20F00100704790F0000F0CF0AE
:104ED800004C08BF49024CEA502040EA51207F3A72
:104EE800C2BFD2F1FF0340EAC250704740F400004D
:104EF8004FF00003013A5DDC12F1190FDCBF00F03E
:104F080000407047C2F10002410021FA02F1C2F1EB
:104F1800200200FA02FC5FEA310040F1000053EA87
:104F28004C0308BF20EADC70704792F0000F00F0D5
:104F3800004C02BF400010F4000F013AF9D040EADB
:104F48000C0093F0000F01F0004C02BF490011F46F
:104F5800000F013BF9D041EA0C018FE70CEAD1536D
:104F680092EA0C0F18BF93EA0C0F0AD030F0004CED
:104F780018BF31F0004CD8D180EA010000F00040A1
:104F8800704790F0000F17BF90F0004F084691F05F
:104F9800000F91F0004F14D092EA0C0F01D1420299
:104FA8000FD193EA0C0F03D14B0218BF084608D162
:104FB80080EA010000F0004040F0FE4040F40000AC
:104FC800704740F0FE4040F4400070474FF0FF0C3F
:104FD8001CEAD0521EBF1CEAD15392EA0C0F93EA86
:104FE8000C0F69D0A2EB030280EA010C49024FEAD8
:104FF800402037D04FF0805343EA111143EA101391
:105008000CF000408B4238BF5B0042F17D024FF448
:10501800000C8B4224BF5B1A40EA0C00B3EB510F23
:1050280024BFA3EB510340EA5C00B3EB910F24BF0C
:10503800A3EB910340EA9C00B3EBD10F24BFA3EB91
:10504800D10340EADC001B0118BF5FEA1C1CE0D159
:10505800FD2A3FF650AF8B4240EBC25008BF20F00C
:10506800010070470CF0004C4CEA50207F32C2BF60
:10507800D2F1FF0340EAC250704740F400004FF0FD
:105088000003013A37E792F0000F00F0004C02BF2E
:10509800400010F4000F013AF9D040EA0C0093F0F8
:1050A800000F01F0004C02BF490011F4000F013B52
:1050B800F9D041EA0C0195E70CEAD15392EA0C0FBA
:1050C80008D142027FF47DAF93EA0C0F7FF470AFF2
:1050D800084676E793EA0C0F04D14B023FF44CAF35
:1050E80008466EE730F0004C18BF31F0004CCAD1CA
:1050F80030F000427FF45CAF31F000437FF43CAF06
:105108005FE700BF42000ED2B2F1FE4F0BD34FF063
:105118009E03B3EB126209D44FEA002343F0004325
:1051280023FA02F070474FF00000704712F1610F48
:1051380001D1420202D14FF0FF3070474FF000001A
:10514800704700BF53B94AB9002908BF00281CBFDF
:105158004FF0FF314FF0FF3000F07AB9ADF1080C95
:105168006DE904CE00F006F8DDF804E0DDE902237D
:1051780004B070472DE9F0478C460E460446089D5A
:10518800002B50D18A4217466CD9B2FA82FEBEF182
:10519800000F0BD0CEF1200C01FA0EF620FA0CFC11
:1051A80002FA0EF74CEA060C00FA0EF43A0CBCFBB5
:1051B800F2F9BBB202FB19CC09FB03FA4FEA144817
:1051C80048EA0C46B2450AD9F61909F1FF3180F0D0
:1051D8002581B24540F22281A9F102093E44A6EB9D
:1051E8000A06B6FBF2F002FB106600FB03F3A4B25A
:1051F80044EA0644A34209D9E41900F1FF3280F0D9
:105208000B81A34240F2088102383C440021E41A91
:1052180040EA0940002D62D0002324FA0EF42C60E5
:105228006B60BDE8F0878B4207D9002D55D000216F
:1052380085E841000846BDE8F087B3FA83F1002904
:1052480040F08F80B34202D3824200F2FC80841A7D
:1052580066EB03060120B446002D40D085E8101007
:10526800BDE8F08712B90127B7FBF2F7B7FA87FE56
:10527800BEF1000F35D10121F61B4FEA174C1FFA7A
:1052880087F8B6FBFCF20CFB126608FB02F0230C55
:1052980043EA0646B04207D9F61902F1FF3302D2B3
:1052A800B04200F2D2801A46361AB6FBFCF00CFB6C
:1052B800106608FB00F8A3B243EA0644A04507D9E4
:1052C800E41900F1FF3302D2A04500F2B980184674
:1052D800A4EB080440EA02409CE729462846BDE8BA
:1052E800F08707FA0EF7CEF1200326FA03F24FEA09
:1052F800174CB2FBFCF11FFA87F80CFB112206FAD7
:105308000EF620FA03F301FB08F933431E0C46EAB4
:105318000246B14500FA0EF409D9F61901F1FF3237
:1053280080F08C80B14540F2898002393E44A6EB7A
:105338000906B6FBFCF00CFB106200FB08F99EB2F4
:1053480046EA0246B14507D9F61900F1FF3371D292
:10535800B1456FD902383E44A6EB090640EA01413F
:105368008FE7C1F1200722FA07F88B4048EA0303C8
:1053780026FA07F44FEA134EB4FBFEF91FFA83FC32
:105388000EFB19448E4020FA07F809FB0CFA48EA8C
:1053980006084FEA184646EA0444A24502FA01F212
:1053A80000FA01F608D9E41809F1FF3044D2A24501
:1053B80042D9A9F102091C44A4EB0A04B4FBFEF08B
:1053C8000EFB104400FB0CFC1FFA88F848EA044462
:1053D800A44507D9E41800F1FF3E29D2A44527D9EE
:1053E80002381C4440EA0940A0FB0289A4EB0C0CDB
:1053F800CC45C246CE4615D312D055B1B6EB0A03FA
:105408006CEB0E0606FA07F7CB401F43CE402F6021
:105418006E600021BDE8F0871046F7E68946DEE6B3
:105428004645EAD2B8EB020A69EB030E0138E4E715
:105438007046D7E718468FE78146BDE7114676E7FD
:1054480002383C4444E7084606E7023A3E442BE764
:10545800704700BF38B50E4B054618784FF47A737D
:10546800B3FBF0F30B4A1068B0FBF3F000F038FB25
:10547800044658B90F2D09D8024629464FF0FF3087
:1054880000F0EEFA044B20461D6038BD012038BDFF
:10549800000000201802002004000020074A08B578
:1054A8001368032043F01003136000F0C7FA0020CC
:1054B800FFF7D0FF03F012F9002008BD00200240DA
:1054C800034A044B11681B780B441360704700BFF4
:1054D8007804002000000020014B1868704700BFC6
:1054E8007804002038B50446FFF7F6FF0546631C2C
:1054F8001EBF044B1B78E418FFF7EEFF401B8442E5
:10550800FAD838BD000000207047436A10B59A6A7F
:1055180012F0500F1BD19A6A42F400729A621A680C
:10552800926802F46022B2F5602F0CD1DA6852B9A1
:105538009A6A22F480729A629A6AD2045EBF9A6A60
:1055480042F001029A621846FFF7DEFF10BD1B6A9F
:10555800BDE810401B6B1847704708B5406AFFF755
:10556800FBFF08BD7047406A08B5836A43F04003F3
:105578008362C36A43F00403C362FFF7F3FF08BD05
:10558800002373B5019390F82430012B74D00123C4
:105598004D6880F82430062D02684FEA85030C68B0
:1055A80025D82B441F25566B053B9D4026EA05054B
:1055B80004FA03F32B435363092C4FEA44038D6821
:1055C8002FD907262344D1681E3B9E4021EA0601B5
:1055D80005FA03F30B43D360A4F11003012B2BD975
:1055E8000023002280F82420184602B070BD0C2D3C
:1055F8000BD82B441F25166B233B9D4026EA050537
:1056080004FA03F32B431363D6E72B441F25D66A0A
:10561800413B9D4026EA050504FA03F32B43D36278
:10562800CAE70726116923449E4021EA060105FAC4
:1056380003F30B431361CFE7104B9A4216D19368DB
:105648001B02CDD49368102C43F400039360C7D198
:105658000B4B0C4A1B68B3FBF2F20A23534301932A
:10566800019B002BBCD0019B013BF8E7836A43F008
:10567800200383620123B4E70223B5E70024014035
:105688001802002040420F00002373B501930368FD
:1056980004469A68D20702D5002002B070BD9A6805
:1056A80042F001029A60124B124A1B68B3FBF2F3F4
:1056B8000193019BC3B9FFF70FFF064623689D6856
:1056C80015F00105E8D1FFF707FF801B0228F5D97F
:1056D800A36A84F8245043F01003A362E36A01200C
:1056E80043F00103E362D8E7019B013BE0E700BF19
:1056F8001802002040420F002DE9D8419046404B47
:10570800026804469A420F4602D03E498A4203D1B3
:105718005B6813F4702F6ED194F82430012B6CD091
:105728000123204684F82430FFF7AEFF0646002800
:105738005DD1A06A216820F47060324B20F001002E
:1057480040F480709942A06204D12D4A536813F442
:10575800702F3ED1A36A23F48013A3624B685A05C5
:1057680005D5A36A23F4405343F48053A362A36A84
:10577800206A13F4805318BFE36A3A4618BF23F02F
:105788000603E362002384F824301F4B4C31836204
:105798001E4BC3621E4B03636FF0020341F84C3C7F
:1057A80051F8443C43F4807341F8443C434600F0CC
:1057B800EDF923689A6802F46022B2F5602F9A68BE
:1057C8000CBF42F4A00242F480129A603046BDE851
:1057D800D881A36A43F48013A36253685B0541BF71
:1057E800A06A20F4405040F48050A062BFE7002334
:1057F80084F82430EAE70126E8E70226E6E700BF56
:105808000024014000280140135500086355000892
:105818006F55000838B5036804469A68D20701D462
:10582800002038BD9A6822F001029A60FFF754FE02
:10583800054623689B68DB07F2D5FFF74DFE401B42
:105848000228F6D9A36A012043F01003A362E36A91
:1058580043F00103E36238BDF8B50446002877D069
:10586800836A23B9C36280F8243002F059FF2046C6
:10587800FFF7D0FFA36A13F010036BD1002869D19A
:10588800A26A374922F4885222F0020242F0020248
:10589800A26294E824008A42E16904D1B1F5402F5C
:1058A80008BF4FF40021E66845EA46052943A56884
:1058B800B5F5807F35D0012D08BF4FF48073676937
:1058C800012F06D17EBBA669013E43EA463343F465
:1058D80000635668B5F5807F26F4694643EA0603F7
:1058E800536096681F4B03EA060343EA010393607B
:1058F80001D0012D20D12369013B1B05D56A25F470
:1059080070052B43D3629268174B1340994215D107
:105918000023E362A36A23F0030343F00103A362B5
:10592800F8BD2B46CBE7A66A46F02006A662E66AD3
:1059380046F00106E662CCE70023DFE7A36A23F01E
:10594800120343F01003A362E36A43F00103E36226
:105958000120F8BDA36A43F01003A362F8E700BF73
:10596800003C0140FDF7E1FFFE0E1FFF002373B569
:10597800019390F824300446012B5AD0012380F873
:105988002430FFF747FF0546002832D1A36A0220DA
:1059980023F4885323F0020343F00203A362264B47
:1059A8001E6800F0AFFFB6FBF0F040000190019BCD
:1059B8001BBB2046FFF768FE2268936843F0080384
:1059C8009360FFF789FD064623689A68120718D482
:1059D8009A6842F004029A60FFF77EFD0646236843
:1059E8009B685B071FD4A36A23F0030343F00103FA
:1059F800A362002384F8243012E0019B013B019349
:105A0800D5E7FFF769FD801B0A28DDD9A36A0125C0
:105A180023F0120343F01003A362002384F8243018
:105A2800284602B070BDFFF757FD801B0A28D6D95B
:105A3800ECE70225F4E700BF18020020074A00023D
:105A4800D36800F4E06023F4E0631B041B0C43F00C
:105A5800BF6343F400330343D360704700ED00E0B5
:105A6800174B30B5DC68C4F30224C4F10703251DC5
:105A7800042B28BF0423062D4FF0010598BF0024EE
:105A880005FA03F303F1FF3388BF033C1940A14033
:105A980005FA04F4013C2240002842EA01024FEAD8
:105AA8000212AFBF00F16040064B00F00F00D2B207
:105AB800A5BFD2B200F561401A5480F8002330BD6A
:105AC80000ED00E014ED00E00123420900F01F00A2
:105AD80003FA00F0014B43F82200704700E100E0B0
:105AE8000138B0F1807F0AD2F021064B064A58608F
:105AF80082F823100020072298601A60704701205E
:105B0800704700BF10E000E000ED00E010B500288D
:105B180032D00168194B1424994225D8184AA3F2A7
:105B280007430A44B2FBF4F2920002648468C36338
:105B380043680A682343C46822F47F5223430469F4
:105B480022F0300223434469234384692343C46910
:105B5800234313430B600122002380F82120836331
:105B680080F82030184610BD064B0B44B3FBF4F305
:105B78009B000364044BD9E7012010BD07040240D1
:105B8800F8FFFDBFF8FBFDBF00040240F0B590F838
:105B98002040012C35D0012490F8215080F8204075
:105BA800A5424FF000064FF0020428D180F82140AA
:105BB800046886632668076C26F001062660C66BB3
:105BC800BD407560636043680568102BC36A0BBFEE
:105BD800A260A160E160E2604BB1236843F00E036C
:105BE80023602B68002043F001032B60F0BD23687D
:105BF80023F004032360236843F00A03F0E780F8E6
:105C080020600220F0BD000090F8213010B5022B72
:105C180003D004238363012010BD03681A6822F0AF
:105C28000E021A601A6822F001021A60294A934289
:105C380024D902F56272934219D01432934218D0D3
:105C48001432934217D0143293420CBF4FF480534E
:105C58004FF48033204A53600123002480F8213018
:105C6800436B80F820409BB39847204610BD012322
:105C7800F0E71023EEE74FF48073EBE717498B4208
:105C880016D014318B4215D014318B4214D01431F4
:105C98008B4214D014318B4214D014318B4214D05F
:105CA800934214BF4FF480334FF080730C4AD2E70D
:105CB8000123FBE71023F9E74FF48073F6E74FF46D
:105CC8008053F3E74FF48033F0E74FF48013EDE7A8
:105CD800184610BD8000024000040240080002403F
:105CE8000000024070B40425C66B026C3468036877
:105CF80095402542196855D04D0753D51A68960620
:105D08005EBF1A6822F004021A60604A93421FD9E3
:105D180002F56272934214D01432934213D01432B3
:105D2800934212D0143293420CBF4FF480434FF485
:105D38008023574A5360C36A002B00F0A58070BCCB
:105D480018470423F5E74023F3E74FF48063F0E7AF
:105D580050498B4216D014318B4215D014318B42E6
:105D680014D014318B4214D014318B4214D0143116
:105D78008B4214D0934214BF4FF480234FF08063BA
:105D8800454AD7E70423FBE74023F9E74FF480634C
:105D9800F6E74FF48043F3E74FF48023F0E74FF43E
:105DA8008003EDE702259540254257D08D0755D54C
:105DB8001A68940606D41A6822F00A021A600122A8
:105DC80080F82120314A93421ED902F5627293422B
:105DD80013D01432934212D01432934211D0143299
:105DE80093420CBF4FF400534FF40033284A5360DA
:105DF800002380F82030836A9EE70223F6E72023F9
:105E0800F4E74FF40073F1E722498B4216D01431BE
:105E18008B4215D014318B4214D014318B4214D0DC
:105E280014318B4214D014318B4214D0934214BFD6
:105E38004FF400334FF00073174AD8E70223FBE70B
:105E48002023F9E74FF40073F6E74FF40053F3E724
:105E58004FF40033F0E74FF40013EDE708259540C1
:105E6800254211D009070FD5196821F00E011960D4
:105E7800012303FA02F27260836380F82130002361
:105E880080F82030036B57E770BC704780000240F1
:105E9800000402400800024000000240114AD36892
:105EA80013F0100305D01049CB6943F00203CB610E
:105EB8001023D268500706D50B4943F00403CA697A
:105EC80042F00102CA61074AD169C90708D50648E4
:105ED800C16941F00401C161D16921F00101D161B9
:105EE800D36070470020024080040020064B1869E8
:105EF80010F0800007D0054A5A6002F188325A60D3
:105F08001869C0F3C010704700200240230167459C
:105F1800034A0020136943F080031361704700BFF0
:105F280000200240F8B50646FFF7D6FA114C07469E
:105F38002546E368D80712D4E368990644BF2023AE
:105F4800E360EB68DA0606D4EB69DB0703D4E8689C
:105F580010F0040002D0FFF7A1FF0120F8BD731C68
:105F6800E7D00EB90320F8BDFFF7B6FAC01B86428A
:105F7800DFD2F7E7002002402DE9F84F1F4C994681
:105F8800237E0546012B0F46904633D001234CF261
:105F980050302376FFF7C6FF40BB012D03D0022DFA
:105FA8000CBF022504250026B246DFF854B03201A2
:105FB80040464946FEF73CF9C4F81CA0DBF810300F
:105FC80080B243F00103CBF8103027F816004CF2EA
:105FD8005030FFF7A7FFDBF8103023F00103CBF8B0
:105FE800103018B90136F3B29D42E0D80023237669
:105FF800BDE8F88F0220BDE8F88F00BF80040020BC
:10600800002002400022064BDA61064B1A6942F072
:1060180004021A611A6942F040021A61704700BF0F
:1060280080040020002002400022064BDA61064B63
:106038001A6942F002021A6158611A6942F0400274
:106048001A61704780040020002002402DE9F041C9
:10605800234D07462B7E8846012B3DD0012403683B
:106068002C76022B4CF2503013D1FFF75BFF20B196
:10607800012000232B76BDE8F081FFF7C3FF4CF227
:106088005030FFF74FFF174A136923F004031361D9
:10609800EFE7FFF747FF0028EAD14FF0FF33C8F8D2
:1060A80000302046BE680F4CFA68BB6803EBC22379
:1060B8009E42DED23046FFF7B7FF4CF25030FFF772
:1060C80031FF236923F00203236110B1C8F800608F
:1060D800CFE706F50066E7E70220BDE8F08100BFDC
:1060E80080040020002002402DE9F74F00221646C8
:1060F8006C4F6D4BDFF8B8E1DFF8B8C14FF001081D
:106108000C6808FA06F808EA0404A04540F08580FF
:106118004D68122D00F0B78000F28D80022D00F03E
:10612800AF8000F28180002D00F09180012D00F0F9
:10613800A5804FF00F09FF2C93BF824606F18045DA
:10614800083DD0F800B092BFB500D0F804B0AD005B
:1061580009FA05F82BEA080802FA05F588BF00F1E4
:10616800040A48EA0505CAF80050D1F804A01AF054
:10617800805F52D0BD6926F0030845F00105BD6176
:10618800BD6908F1804805F00105019508F58038DA
:1061980006F0030B019D4FEA8B0BD8F8085009FA5B
:1061A8000BF925EA0909414DA84271D005F580652A
:1061B800A8426FD005F58065A8426DD005F58065C9
:1061C800A8426BD005F58065A84269D070450CBF20
:1061D8000525062505FA0BF545EA0905C8F808500E
:1061E8001D681AF4803F14BF2543A5431D605D68F0
:1061F8001AF4003F14BF2543A5435D609D681AF457
:10620800801F14BF2543A5439D60DD681AF4001F55
:1062180014BF2C4325EA0404DC600136102E7FF4F9
:106228006DAF03B0BDE8F08F032D25D0112D80D1BF
:10623800CA6804327DE7654509D012D8DFF878903E
:106248004D4504D009F580394D457FF472AF8A6811
:10625800E2B1012A0CBFC0F81080C0F814800822EF
:1062680067E7DFF858904D45F1D009F580394D457D
:10627800EDD0A9F58019E7E700225AE7CA6858E780
:10628800CA68083255E7CA680C3252E7042250E758
:1062980000259FE701259DE702259BE7032599E750
:1062A800042597E70010024000040140000801405F
:1062B800001C0140000021100000111000003110E6
:1062C8008368194214BF0120002070470AB1016198
:1062D80070470904FBE7C3685940C1607047000074
:1062E80003682DE9F341DB07054610D42B689F07A7
:1062F8005ED42B68190700F195802B685A0700F1C6
:10630800BF80EA69002A40F02D81002014E0904CFB
:10631800636803F00C03042B07D0636803F00C03D5
:10632800082B0CD16368DE0309D523689C03DDD5EF
:106338006B68002BDAD1012002B0BDE8F0816B68F0
:10634800B3F5803F10D1236843F480332360FFF70F
:10635800C3F8064623689803C8D4FFF7BDF8801B26
:106368006428F7D90320E7E79BB9236823F480332F
:106378002360236823F480232360FFF7ADF80646E3
:1063880023689903B2D5FFF7A7F8801B6428F7D9CB
:10639800E8E7B3F5A02F236803D143F480232360F3
:1063A800D1E723F480332360236823F48023CDE7E7
:1063B800674C636813F00C0F07D0636803F00C0395
:1063C800082B10D16368DA030DD423689B0702D524
:1063D8002B69012BAFD123686A6923F0F80343EADC
:1063E800C203236085E72A695A4B6AB101221A6001
:1063F800FFF772F8064623689F07ECD4FFF76CF89E
:10640800801B0228F7D9ADE71A60FFF765F8064642
:10641800236898077FF56DAFFFF75EF8801B0228A9
:10642800F6D99FE7AA694A4C4B4BDAB101221A60A8
:10643800FFF752F80646636A9B070DD54FF4FA52E8
:10644800464B1B68B3FBF2F3019300BF019B5A1E36
:106458000192002BF9D150E7FFF73EF8801B022884
:10646800E9D97FE71A60FFF737F80646636A9F079E
:106478007FF543AFFFF730F8801B0228F6D971E7A4
:10648800334CE369D80024D40127E36943F08053EF
:10649800E361E36903F080530093009B304E336857
:1064A800D90518D5EB68012B26D1236A43F00103DF
:1064B8002362FFF711F841F288368046236A9B076A
:1064C8003FD5002F3FF41DAFE36923F08053E3610C
:1064D80017E70027E2E7336843F480733360FEF779
:1064E800FBFF80463368DA05DCD4FEF7F5FFA0EB46
:1064F80008006428F6D935E7ABB9236A41F2883831
:1065080023F001032362236A23F004032362FEF7C6
:10651800E3FF0646236A9807D3D5FEF7DDFF801B05
:106528004045F7D91EE7052B236A03D143F004033E
:106538002362BAE723F001032362236A23F00403EA
:10654800B6E7FEF7C9FFA0EB0800B042B6D909E7E5
:10655800001002400000424280044242180200201B
:1065680000700040224C636803F00C03082B3FF4D2
:10657800E2AE00231F4E022A33602BD1FEF7ACFF98
:106588000746236899011FD42B6AB3F5803F05D1CC
:106598006268A96822F400320A436260696A626824
:1065A8000B4322F474121343636001233360FEF734
:1065B80093FF054623689A013FF5A7AEFEF78CFFC7
:1065C800401B0228F6D9CDE6FEF786FFC01B02283D
:1065D800D7D9C7E6FEF780FF054623689B017FF5FC
:1065E80094AEFEF779FF401B0228F6D9BAE600BF41
:1065F800001002406000424230B5194B87B002AC2F
:1066080003F11005224618685968083303C2AB42E3
:106618001446F7D101238DF80430022311498DF86F
:1066280005304B6803F00C02082A17D1C3F38342E4
:1066380006A80244DB0312F8102C0CD54B680A4854
:10664800C3F34043504306AA134413F8143CB0FB69
:10665800F3F007B030BD05485043FAE70248F8E7C1
:1066680000C000080010024000127A0000093D0036
:10667800544A2DE9F0411368054603F007038B429D
:106688000E462AD329688C0734D4CA0747D44D4A02
:10669800136803F007039E42C0F082802A684A4CC0
:1066A80012F0040F40F08780130706D563682A6943
:1066B80023F4605343EAC2036360FFF79DFF6368F6
:1066C800424AC3F30313D35CD840414B18600020FF
:1066D800FEF7C0FE0020BDE8F081136823F0070331
:1066E8000B431360136803F007039942CAD00120D3
:1066F800BDE8F081344B11F0040F1EBF5A6842F414
:10670800E0625A60080742BF5A6842F460525A6011
:106718005A68A86822F0F00202435A60B5E76A682E
:10672800294C012A23681CD113F4003FDFD0636889
:1067380041F2883823F0030313436360FEF7CCFE6D
:106748006B680746012B14D1636803F00C03042B14
:106758009DD0FEF7C1FEC01B4045F5D90320BDE81A
:10676800F081022A02D113F0007FDFE713F0020F55
:10677800DCE7022B0FD1636803F00C03082B86D0EB
:10678800FEF7AAFEC01B4045F5D9E7E7FEF7A4FED1
:10679800C01B4045E2D8636813F00C0FF6D176E7CA
:1067A800136823F0070333431360136803F00703E8
:1067B8009E429CD172E76368E96823F4E0630B4367
:1067C800636071E700200240001002403FC00008EB
:1067D80018020020044B054A5B68C3F30223D35C0C
:1067E800034A1068D8407047001002404FC00008A4
:1067F80018020020044B054A5B68C3F3C223D35C2C
:10680800034A1068D8407047001002404FC0000883
:106818001802002003682DE9F341D907054620D561
:10682800354CE369DA0032D40127E36943F0805339
:10683800E361E36903F080530193019B2F4E3368B2
:10684800DB0526D5236A13F4407336D1236A6A68B8
:1068580023F44073134323621FB1E36923F0805389
:10686800E3612868830706D5234AA968536823F497
:1068780040430B43536010F010001BD01E4A696957
:106888005368002023F480030B43536012E0002771
:10689800D4E7336843F480733360FEF71DFE804607
:1068A8003368D805CED4FEF717FEA0EB080064289D
:1068B800F6D9032002B0BDE8F0816A6802F440729C
:1068C8009342C3D001200E4A236A1060002023F4AB
:1068D800407110602162D907B8D5FEF7FDFD41F27D
:1068E80088380646236A9A07B0D4FEF7F5FD801B60
:1068F8004045F7D9DDE700BF0010024000700040B6
:1069080040044242024670B53B4B86B002AD03F1EB
:1069180010062C4618685968083303C4B342254644
:10692800F7D101238DF804300223501E8DF805306D
:106938000F285ED8DFE800F032515D2D5D5D5D2DDA
:106948005D5D5D5D5D5D5D082C4B5968186810F0F4
:10695800807037D0C1F3834206A8024412F8100CA5
:10696800CA0341BF5A6806A9C2F34042521844BF3D
:1069780012F8141C224A5B684CBFB2FBF1F2214AA0
:106988005B0202FB00F01DD403234000B0FBF3F0D0
:1069980018E006B0BDE87040FFF72EBE40F20231A5
:1069A800164A136A1940B1F5817F1FD003F440736A
:1069B800B3F5007F08D149F64040536A13F0020F3F
:1069C80008BF002006B070BDB3F5407F11D1136831
:1069D8004FF2244013F4003FF2E7FFF70BFF074B99
:1069E8005B68C3F3813301335B00CFE74FF40040AA
:1069F800E8E70020E6E700BF10C0000800100240EA
:106A080000127A0000093D007047704770477047D0
:106A1800036810B51A69044691070ED5DA6892071B
:106A28000BD56FF002021A6101229B6902779B075E
:106A380077D0FFF7EAFF0023237723681A69500706
:106A480010D5DA6851070DD56FF004021A610222D9
:106A58009B69227713F4407F204668D0FFF7D5FF63
:106A68000023237723681A6912070FD5DA681007FD
:106A78000CD56FF008021A610422DB6922779907A6
:106A880020465AD0FFF7C1FF0023237723681A69ED
:106A9800D20610D5DA68D0060DD56FF010021A614B
:106AA8000822DB69227713F4407F20464BD0FFF79A
:106AB800ACFF0023237723681A69D10708D5DA6861
:106AC800D20705D56FF0010220461A6101F09AFA43
:106AD80023681A69100608D5DA68110605D56FF01B
:106AE800800220461A6100F0BEF823681A6952062F
:106AF80008D5DA68500605D56FF0400220461A61BD
:106B0800FFF785FF23681A69910622D5DA6892068D
:106B18001FD56FF020022046BDE810401A6100F032
:106B2800A1B8FFF771FF2046FFF770FF83E7FFF773
:106B38006BFF2046FFF76AFF92E7FFF765FF2046E5
:106B4800FFF764FFA0E7FFF75FFF2046FFF75EFF50
:106B5800AFE710BD244A0368904212D002F50062E4
:106B680090420ED0B0F1804F0BD0A2F598329042EF
:106B780007D002F58062904203D002F5806290420D
:106B88001DD14A6823F070031343174A904212D06C
:106B980002F5006290420ED0B0F1804F0BD0A2F502
:106BA8009832904207D002F58062904203D002F5F5
:106BB8008062904203D1CA6823F4407313434A6940
:106BC80023F08003134303608B68C3620B688362FE
:106BD800054B984203D003F50063984201D10B6935
:106BE8000363012343617047002C014010B504463C
:106BF800A0B190F83D3003F0FF021BB980F83C20AB
:106C080001F0FEFD0223206884F83D30211DFFF7C6
:106C1800A1FF0123002084F83D3010BD012010BDE4
:106C280090F83C3010B5012B4FF0020318D080F8D3
:106C38003D3003680C685A68496822F070025A604F
:106C48005A6822435A609A6822F080029A609A68C9
:106C58000A439A60012380F83D30002380F83C30D5
:106C6800184610BD704770470368DA6822F49072BE
:106C7800DA605A6922F001025A61202380F83A301A
:106C8800704700002DE9F0470568C2682B69016963
:106C980023F4405313432B618368EA680B4341692B
:106CA80022F4B05222F00C020B431343EB606B69E1
:106CB800826923F4407313436B61404B81469D42C4
:106CC8004FF0190446D1FFF795FD04FB00F3D9F8FE
:106CD80004604FF06408B600B3FBF6F3B3FBF8F3B7
:106CE8001E01FFF787FD6043D9F804309B00B0FB15
:106CF800F3F7FFF77FFD6043D9F804309B00B0FB42
:106D0800F3F3B3FBF8F308FB13731B013233B3FB44
:106D1800F8F303F0F007FFF76DFD6043D9F804209E
:106D28009200B0FBF2FAFFF765FD6043D9F8043032
:106D38009B00B0FBF3F3B3FBF8F308FB13A31B01B1
:106D48003233B3FBF8F303F00F033B433344AB6038
:106D5800BDE8F087FFF73EFD04FB00F3D9F80460B7
:106D68004FF06408B600B3FBF6F3B3FBF8F31E016B
:106D7800FFF730FD6043D9F804309B00B0FBF3F710
:106D8800FFF728FD6043D9F804309B00B0FBF3F30C
:106D9800B3FBF8F308FB13731B013233B3FBF8F3AF
:106DA80003F0F007FFF716FD6043D9F804209200BE
:106DB800B0FBF2FAFFF70EFDB7E700BF003801405D
:106DC800F8B504460E4617461D4621680B6836EA94
:106DD800030301D10020F8BD6B1CF7D095B92368D7
:106DE8000320DA6822F4D072DA605A6922F00102CC
:106DF8005A61202384F8393084F83A30002384F823
:106E08003830F8BDFEF768FBC01B8542DDD2E6E7E7
:106E180010B5044640B390F8393003F0FF021BB9AF
:106E280080F8382001F000FD2423226884F83930E6
:106E3800D368204623F40053D360FFF723FF236869
:106E480000201A6922F490421A615A6922F02A0233
:106E58005A61DA6842F40052DA602023E06384F869
:106E6800393084F83A3010BD012010BD2DE9F041C9
:106E78001F4690F839300446202B0D4690464ED1D7
:106E8800002949D0002A47D090F83830012B46D045
:106E9800012380F838300023C363212380F8393078
:106EA800FEF71AFB0646A4F82480A4F82680E38C93
:106EB8009BB26BB93B46324640212046FFF780FF24
:106EC800A8B9202384F8380084F83930BDE8F08167
:106ED800E38C3246013B9BB2E384A3688021B3F57F
:106EE800805F20463B460ED1FFF76AFF10B10320B2
:106EF800BDE8F0812B882268C3F308035360236937
:106F080043B90235D3E7FFF75BFF0028EFD12368C9
:106F18002A785A600135CAE70120BDE8F0810220CD
:106F2800BDE8F08138B50446134694F83920202A84
:106F38002AD139B333B394F83820012A24D0012256
:106F4800002584F838202122E384206BE56384F847
:106F580039200E4AA384216282620D4A4563C262C7
:106F68000C4A026322680432FEF710FE6FF04002FA
:106F7800236828461A605A6984F8385042F080021B
:106F88005A6138BD012038BD022038BD3370000871
:106F9800617000082D710008134690F83A2073B507
:106FA800202A054638D1002934D0002B32D090F859
:106FB8003820012A30D00122002480F838202222EB
:106FC80081628385C46380F83A20406B134A2E6837
:106FD8008262134A4463C262124A02630A46311D3E
:106FE800FEF7D4FD20462B6801941A6801925A686E
:106FF80085F838400192019ADA6842F48072DA60C2
:107008005A6942F001025A615A6942F040025A61D3
:1070180002B070BD0120FBE70220F9E76B700008A1
:10702800217100082D710008704708B50368426A8D
:107038001B6813F020030AD1D38413685A6922F01D
:1070480080025A61DA6842F04002DA6008BD1046F0
:10705800FFF7EAFF08BD704708B5406AFFF7FBFF76
:1070680008BD08B50368426A1B6813F0200310D1F5
:10707800D3851368D96821F48071D960596921F0E2
:1070880001015961596921F040015961202382F8B1
:107098003A30104601F006FD08BD90F83A3010B5B8
:1070A800222B36D183680169B3F5805F0268836A51
:1070B80023D15268E9B9C2F3080223F8022B83628C
:1070C800C48D013CA4B2C4858CB90368DA6822F087
:1070D8002002DA60DA6822F48072DA605A6922F0F3
:1070E80001025A61202380F83A3001F0DBFC0020CD
:1070F80010BDD2B223F8012BE1E721B9591C52681F
:1071080081621A70DCE75268591C816202F07F02C2
:10711800F7E7022010BD704708B5406AFFF7FBFF8C
:1071280008BD7047416A08B50B685A6991F839007B
:1071380021280AD1120608D50022CA84DA6822F06A
:10714800C002DA60202281F839205B6991F83A2080
:10715800222A06D15B0604D500230846CB85FFF713
:1071680083FDCB6B084643F01003CB63FFF7D9FFD1
:1071780008BD0000036870B51A6804461607D96888
:107188005D6907D196065AD58D0658D5BDE8704079
:10719800FFF783BF15F0010502D111F4907F4ED09F
:1071A800D30705D5CE0542BFE36B43F00103E36384
:1071B800500704D51DB1E36B43F00203E363930763
:1071C80004D51DB1E36B43F00403E363160704D54C
:1071D8001DB1E36B43F00803E363E36B002B66D058
:1071E800950604D5880602D52046FFF756FF236882
:1071F80020465D69E26B110702D415F040051AD0EC
:10720800FFF732FD23685A69520610D55A69606B38
:1072180022F040025A6150B1254B4363FEF7F4FC5B
:10722800002844D0606BBDE87040436B1847204687
:10723800FFF777FF70BDFFF774FFE56370BD1606B3
:1072480027D50D0625D594F83920212A2FD1A268F3
:10725800B2F5805F226A17D11188C1F3080159601D
:10726800216979B902322262E28C013A92B2E2844F
:10727800EAB9DA6822F08002DA60DA6842F040029D
:10728800DA6070BD0132EEE7511C216212785A6053
:10729800EAE750060BD54A0609D5DA68204622F0F7
:1072A8004002DA60202384F83930FFF7BDFE70BD54
:1072B800BD72000808B50023406AC385C384FFF780
:1072C80030FF08BD70B50022054604212448FEF7AA
:1072D800FDFF1024224E012208213046FEF7F6FF5A
:1072E8002B044CBF0122002210213046FEF7EEFF8E
:1072F800013C002208213046FEF7E8FF6D0014F03B
:10730800FF04ADB2E7D101224FF400411548FEF762
:10731800DDFF0A2000F018FE22464FF40041114814
:10732800FEF7D4FF012204210D48FEF7CFFF2246C5
:1073380010210B48FEF7CAFF01224FF4004109480B
:10734800FEF7C4FF224604210548FEF7BFFF224688
:10735800BDE870404FF400410248FEF7B7BF00BFD8
:10736800002001400014014008B548F20C00FFF766
:10737800A9FF4FF42040FFF7A5FF40F6FF70FFF785
:10738800A1FF41F2FF30FFF79DFF42F2FF40FFF7F8
:1073980099FF43F2FF50FFF795FF44F2FF60FFF7B4
:1073A80091FF45F2FF70FFF78DFF46F6FF00FFF7EC
:1073B80089FF47F6FF10FFF785FFBDE80840012069
:1073C800FEF790B884B02DE9F84F0AAC84E80F00B6
:1073D8000E9EBDF83C7000223946814630469DF825
:1073E8004050BDF82CA0DDF83080BDF834B0FEF771
:1073F8006DFF0120FEF776F8062415F0010218BF8C
:10740800012259464046FEF761FF0122514648468F
:10741800FEF75CFF0120FEF765F80022514648465A
:10742800FEF754FF013C0120FEF75CF814F0FF045E
:107438004FEA5505E1D1224651464846FEF746FF38
:1074480022464FF480614046FEF740FF0120FEF7D8
:1074580049F8394601223046FEF738FF0120FEF789
:1074680041F8224639463046BDE8F84F04B0FEF7E9
:107478002DBF00001FB50024424B029403F11002F7
:1074880092E803008DE803000FCBFFF79BFF3E4B0C
:10749800029403F1100292E803008DE803000FCB79
:1074A800FFF790FF394B029403F1100292E80300B2
:1074B8008DE803000FCBFFF785FF354B029403F1EE
:1074C800100292E803008DE803000FCBFFF77AFF64
:1074D800304B029403F1100292E803008DE8030098
:1074E8000FCBFFF76FFF2C4B029403F1100292E8C9
:1074F80003008DE803000FCBFFF764FF274B0294CE
:1075080003F1100292E803008DE803000FCBFFF7A8
:1075180059FF234B029403F1100292E803008DE80F
:1075280003000FCBFFF74EFF1E4B029403F110022E
:1075380092E803008DE803000FCBFFF743FF1A4BD7
:10754800029403F1100292E803008DE803000FCBC8
:10755800FFF738FF154B029403F1100292E803007D
:107568008DE803000FCBFFF72DFF114B029403F1B9
:10757800100292E803008DE803000FCBFFF722FF0B
:1075880004B010BD080000202000002038000020B2
:107598005000002068000020800000209800002093
:1075A800B0000020C8000020E0000020F800002003
:1075B8001001002010B5FF230446221AD2B29142CE
:1075C80001D8184610BD14F8012B5340082213F0B7
:1075D800800F02F1FF324FEA430318BF83F03103F3
:1075E80012F0FF02DBB2F2D1E7E730B5FF23054620
:1075F8002C1AE4B2A14203D89B1A5842584130BD14
:1076080015F8014B6340082413F0800F04F1FF3490
:107618004FEA430318BF83F0310314F0FF04DBB2D1
:10762800F2D1E5E784B08DE80F009DF818209DF8A9
:107638001C3002981A4112F00102BDF80C1018BF54
:10764800012204B0FEF742BE84B02DE9F04F85B0A8
:107658000EAC84E80F00129DBDF84C600022314644
:1076680080462846BDF83C90FEF730FE0A2000F020
:107678006BFC00270DF1480B0DF1640A9DF85030A2
:10768800FCB202931295ADF84C6003949BE803009A
:107698008DE80300CDF83880ADF83C900EAB0FCBE9
:1076A800FFF7C0FF9DF86C30039402939AE803003B
:1076B8008DE8030015AB0FCBFFF7B4FF9DF88830BA
:1076C8000394029320AB93E803008DE803001CABFE
:1076D8000FCBFFF7A7FF9DF8A4300394029327ABC5
:1076E80093E803008DE8030023AB0FCBFFF79AFF65
:1076F8009DF8C030039402932EAB93E803008DE805
:1077080003002AAB0FCBFFF78DFF9DF8DC30039405
:10771800029335AB93E803008DE8030031AB0FCB40
:10772800FFF780FF012249464046FEF7CFFD0A20B9
:1077380000F00AFC0137002249464046FEF7C6FD24
:10774800082F9BD100224FF400410A48FEF7BEFDE6
:10775800314601222846FEF7B9FD0A2000F0F4FB65
:1077680000223146284605B0BDE8F04F04B0FEF7C8
:10777800ADBD00BF000C0140F0B5274C274E254693
:107788000FCE0FC596E80300254F04F11C0685E8C7
:1077980003000FCF0FC697E80300224F86E80300C7
:1077A8000FCF04F138060FC697E803001E4F86E88E
:1077B80003000FCF04F154060FC697E803001B4FD0
:1077C80086E803000FCF04F170060FC697E80300A0
:1077D800174F86E803000FCF04F18C060FC697E811
:1077E80003000023A7B086E80300982229466846CC
:1077F800237684F8343084F8503084F86C3084F878
:10780800883084F8A43001F079FF94E80F00FFF77E
:107818001BFF27B0F0BD00BFD8040020880100205E
:107828005801002028010020A0010020700100203C
:107838004001002070B50223044601250020E60718
:1078480048BF05FA03F603F1010348BF80190E2B60
:107858004FEA5404F3D10124CD0748BF04FA03F5D5
:1078680003F1010348BF4019162B4FEA5101F3D128
:10787800D30748BF00F5800070BDF0B5064601206B
:10788800022407469DF8145016F0010F18BF07FA96
:1078980004FE04F1010418BF70440E2C4FEA56068A
:1078A800F2D10126CF0748BF06FA04F704F1010414
:1078B80048BFC019122C4FEA5101F3D1D70744BF72
:1078C80000F580201324DE0742BF012303FA04F4E5
:1078D8000019EC0748BF00F500209DF81830A907EB
:1078E80048BF00F580106A0748BF00F50010DB07A5
:1078F80048BF00F58000F0BD2DE9F74F16464FF45C
:107908007A729DF838B0002502FB0BF28246DDE959
:107918000C011F46D317FDF715FC0F9A2B4680461E
:107928008946FDF70FFCC0EB40144FF47A72002330
:1079380000EB840439463046FDF704FCFCF706FEEC
:107948004FF47A7206460F46002340464946FDF733
:10795800F9FBFCF7FBFD02460B4630463946FCF7BF
:1079680055FF00221A4BFCF751FF0F460646FDF75C
:10797800FBF81FFA80F84046FCF7A8FD0B460246C4
:1079880039463046FCF764FCFDF70EF9E400A4B272
:1079980006462046FDF712FA01463046FDF762FA20
:1079A800FDF7B0FB2A46414680B2FFF743FF0223AA
:1079B8000646009301952B46012259462046FFF7BB
:1079C8005CFF8AE84100504603B0BDE8F08F00BF75
:1079D80000408F400E4B9A7F4AB9DA7F3AB993F844
:1079E800202022B98722DA775F2283F8202093F8B3
:1079F80021205AB993F8222042B993F823202AB9B2
:107A0800992283F82220B12283F82320704700BFEF
:107A18008005002084B02DE9F04F85B00EAC84E8D5
:107A28000F00179BBDF83C80C3F30A0ABDF8583015
:107A3800109C0193159BBDF8445023F07F4302939B
:107A4800149B129E23F07F43BDF84C7000224146E0
:107A580003938146FEF73AFC002229462046FEF7AA
:107A680035FC002239463046FEF730FC4FF00B0B50
:107A78001AF4806218BF012229462046FEF726FC28
:107A8800322000F061FA012241464846FEF71EFC0A
:107A9800322000F059FA002241464846FEF716FC0B
:107AA800BBF1010B4FEA4A0AE2D1012239463046BE
:107AB800FEF70CFC322000F047FA5A4639463046A9
:107AC800FEF704FC4FF0100A019B294613F400420C
:107AD80018BF01222046FEF7F9FB322000F034FAE5
:107AE800012241464846FEF7F1FB322000F02CFA0D
:107AF800002241464846FEF7E9FB019BBAF1010A1C
:107B08004FEA43039BB20193DED101223946304646
:107B1800FEF7DCFB322000F017FA524639463046B1
:107B2800FEF7D4FB4FF0180A029B294613F4000213
:107B380018BF01222046FEF7C9FB322000F004FAE4
:107B4800012241464846FEF7C1FB322000F0FCF90D
:107B5800002241464846FEF7B9FB029BBAF1010AEA
:107B68004FEA430323F07F430293DDD101223946D4
:107B78003046FEF7ABFB322000F0E6F952463946B4
:107B88003046FEF7A3FB4FF0180A039B294613F46F
:107B9800000218BF01222046FEF798FB322000F0B1
:107BA800D3F9012241464846FEF790FB322000F007
:107BB800CBF9002241464846FEF788FB039BBAF101
:107BC800010A4FEA430323F07F430393DDD1524672
:107BD80029462046FEF77AFB394601223046FEF751
:107BE80075FB322000F0B0F952463946304605B0F0
:107BF800BDE8F04F04B0FEF769BB000038B50023BC
:107C08001A4CBE2223601A4B0546A3600123E36089
:107C180043706023837061230270C370FEF766F9B6
:107C280014492046FEF712FA18B1134802F04EFA2A
:107C3800FEE704462B195B782A5D04F1006102EB2C
:107C4800032292B2002301F5FF210120FEF794F9E7
:107C580020B1A521094802F0C5F9FEE70234642CD9
:107C6800E8D1BDE83840FEF753B900BF3C04002016
:107C780000F807084C04002020C000082EC00008A7
:107C880008B5FFF7BBFF012008BD002303F1006220
:107C980002F5FF221188C1541288C1180233C2F3B9
:107CA8000722642B4A70F1D10120704770B5244D2A
:107CB8004FF480412846FEF703FB224C4FF4004165
:107CC80084F843002846FEF7FBFA1F4E84F8440068
:107CD80001213046FEF7F4FA022184F845003046C7
:107CE800FEF7EEFA802184F846001848FEF7E8FA15
:107CF80006F5006684F84A004FF400713046FEF736
:107D0800DFFA4FF4806184F849003046FEF7D8FA6C
:107D18004FF4006184F847003046FEF7D1FA4FF47B
:107D2800805184F848002846FEF7CAFA4FF480616B
:107D380084F84B002846FEF7C3FA84F84C0070BD5F
:107D480000100140E3050020001801400014014024
:107D5800433810B50C460D2877D8DFE800F0071235
:107D68001920353C2D26434A5151515139B1012230
:107D78004FF480413548BDE81040FEF7A7BA0A46DF
:107D8800F6E719B101224FF40041F3E70A46FAE792
:107D980019B1012201212E48EDE70A46FAE711B18F
:107DA80001220221F7E70A46FBE719B101228021E7
:107DB8002848E0E70A46FAE721B101224FF40071AA
:107DC8002548D8E70A46F9E719B101224FF480613E
:107DD800F6E70A46FAE719B101224FF40061EFE726
:107DE8000A46FAE719B101224FF48051C2E70A4660
:107DF800FAE719B101224FF48061BBE70A46FAE7B6
:107E080091B1002220211448FEF760FA0022402197
:107E18001148FEF75BFA012280210F48FEF756FA57
:107E280001224FF48071CBE7012220210A48FEF796
:107E38004DFA012240210848FEF748FA22468021DF
:107E48000548FEF743FA2246EBE710BD0010014053
:107E580000180140001401400020014010B5074CF3
:107E6800A178601CFFF7A6FB84F86100204601F0AA
:107E7800A7FBBDE8104000F04BBE00BF8005002006
:107E880070B52E4D2E4C284600228021FEF71EFA92
:107E9800204600224FF40071FEF718FA204600220F
:107EA8004FF48061FEF712FA204600224FF4006179
:107EB800FEF70CFA28460022A5F580658021FEF71A
:107EC80005FA204E284600224FF48051FEF7FEF9AD
:107ED800284600224FF48061FEF7F8F93046002268
:107EE8000121FEF7F3F9304600220221FEF7EEF9F0
:107EF800284600224FF48041FEF7E8F92846002280
:107F08004FF40041FEF7E2F9204600222021FEF757
:107F1800DDF9204600224021FEF7D8F9204601224B
:107F28008021FEF7D3F9204601224FF48071FEF735
:107F3800CDF9BDE870400120FDF7D4BA0014014026
:107F48000020014000180140084A0949126882B01F
:107F5800B2FBF1F20190019B53430193019B5A1E1E
:107F68000192002BFAD102B0704700BF180200201E
:107F780040420F0010B5064C2368B3F5FA7F06D9C6
:107F88004FF480410348FEF7A6F90023236010BD93
:107F9800580400200020014040F6C4120B4BF0B5F5
:107FA800196891421A460FD900231C46084F094EFA
:107FB80057F8130099190233050A1C2B81F825502C
:107FC80081F826001460F3D1F0BD00BF50040020F2
:107FD800A0040020E305002070B5074D074C084EAB
:107FE800AB68002B02DD2368642B00D870BD3046D7
:107FF80000F028FDF4E700BFC40B00205C0400205B
:108008000007002002680A4B9A420FD1094A1368F8
:1080180001331360084A136801331360074A136871
:1080280001331360064A136801331360704700BFB9
:10803800001000405C040020580400205004002078
:108048005404002010B514460A230248FEF70EFF18
:10805800204610BD0007002010B596B02822002148
:108068000CA801F056FB1422002101A801F051FBD5
:10807800182200210DEB020001F04BFB01231093A5
:108088001023022411934FF440130CA815930C9459
:108098001394FEF725F90F234FF480620193002310
:1080A800214601A80393049205930294FEF7E0FA8F
:1080B8004FF4804306A806940893FEF7ABFB16B06E
:1080C80010BD000080B5B04D8CB0FDF7E7F9FFF7A3
:1080D800C3FF1022002108A801F01BFBAB69002296
:1080E80043F04003AB61AB697F2103F04003019388
:1080F800019BAB69A54843F01003AB61AB69002451
:1081080003F010030293029BAB69012643F080033E
:10811800AB61AB69022703F080030393039BAB6950
:108128004FF00C0943F00403AB61AB694FF00E0844
:1081380003F004030493049BAB694FF0070A43F070
:108148000803AB61AB6903F008030593059BAB69B2
:1081580043F02003AB61AB6903F020030693069B51
:10816800AB6943F48073AB61AB6903F48073079325
:10817800079BFEF7ABF800224FF6C0418448FEF794
:10818800A5F8002240F2F3318248FEF79FF800225A
:1081980048F6FF718048FEF799F8002247F6FC710F
:1081A8007E48FEF793F800224FF400417C48FEF722
:1081B8008DF8002218217B48FEF788F87F2308A94C
:1081C8007248089309960B970A94FDF78DFF4FF6AE
:1081D800C04308A96E48089309960B970A94FDF7BF
:1081E80083FF40F2F33308A96A48089309960B976E
:1081F8000A94FDF779FF08A96648CDF820900994FC
:108208000A94FDF771FF48F6FF7308A962480893BE
:1082180009960B970A94FDF767FF4FF4405308A996
:108228005D48089309940A94FDF75EFF47F6FC73CE
:1082380008A95A48089309960B970A94FDF754FF22
:108248004FF4407308A95248089309940A94FDF71B
:108258004BFF4FF4004308A95148089309960B9720
:108268000A94FDF741FF182308A94E480893099678
:108278000B970A94FDF738FF602308A9494808932B
:1082880009940A94FDF730FF6B6933436B616B699E
:10829800454D33400093009B444B28462B604FF4D8
:1082A8008073AB604FF46023EE60EB61089409942F
:1082B8000A946C616C60C5F81080FDF7CDFA08A9C6
:1082C80028460996CDF828A00894FDF759F908968C
:1082D800032608A928460997FDF752F908A9284650
:1082E80008970996FDF74CF90896042608A9284628
:1082F8000996FDF745F90896052608A9284609961E
:10830800FDF73EF90896062608A928460996FDF7BE
:1083180037F90896082608A92846CDF824A0FDF7BD
:108328002FF908A92846CDF820A00996FDF728F9C5
:10833800089609264FF00A0A0B2708A92846099625
:10834800FDF71EF908960D2608A92846CDF824A0A1
:10835800FDF716F908A92846CDF820A00997FDF7DA
:108368000FF908A928460897CDF82490FDF708F9D1
:1083780008A928460996CDF82090FDF701F908A923
:108388002846089614E000BF00100240001801407B
:1083980000100140001C0140001401400020014071
:1083A80000080140000C01408C0600200024014018
:1083B800CDF82480FDF7E4F84FF4E1333848394A22
:1083C800846080E80C00C4600461C0F81490846183
:1083D800C461FEF71DFD41F2DF53334E3349304689
:1083E80086E80A0008940994B460C6F80CA0B46141
:1083F800FEF7FCFB08A9304608940994FEF710FC28
:10840800224621462520FDF72BFB2520FDF75CFBA6
:10841800224621463620FDF723FB3620FDF754FB84
:10842800224621463846FDF71BFB3846FDF74CFB34
:10843800224621464046FDF713FB4046FDF744FB24
:10844800224621460F20FDF70BFB0F20FDF73CFBD2
:10845800174800F0D7FAFFF713FDFFF727FC284667
:10846800FDF784FA0028FAD1FEF77EFF1148FFF7DE
:108478000CFCFFF7AFFA00F025F8FFF77DF9FEF7DF
:10848800F9FFFFF7EBFC0E220B490C48FDF734F916
:10849800FFF770FDFFF7A0FDFFF77EFDF8E700BFCF
:1084A8000007002000380140840700200010004029
:1084B800C40B002080050020A00400208C060020AA
:1084C80070470000104B9A7D2AB9DA7D1AB93E220E
:1084D8009A758022DA751A7E2AB95A7E1AB9382214
:1084E8001A76D6225A769A7E2AB9DA7E1AB94D2297
:1084F8009A76EE22DA761A7F2AB95A7F1AB9592261
:108508001A77A6225A77704780050020012370B594
:1085180002241D46C60748BF05FA04F604F1010403
:1085280048BF9B19082C4FEA5000F3D10120CD0712
:1085380048BF00FA04F504F1010448BF5B19152C83
:108548004FEA5101F3D1D20748BF03F5001318468B
:1085580070BD00004CF25033B0FBF3F3372B09D950
:1085680005490022B0FBF1F1A3EB411080B289B2BA
:10857800FFF7CCBF04207047006A180084B02DE9CB
:10858800F74F0CAC84E80F00139BBDF8347023F050
:108598007F430193129BDDF83880BDF83C9023F0AF
:1085A8007F43109DBDF844600022394600938246FF
:1085B800149CFDF78BFE002249464046FDF786FED7
:1085C800002231462846FDF781FE4FF0180B24F0B3
:1085D8007F4414F4000218BF012249464046FDF7C3
:1085E80075FE012239465046FDF770FE0A20FFF756
:1085F800ABFC002239465046FDF768FE6400BBF12B
:10860800010B24F07F44E4D1012231462846FDF7CE
:108618005DFE0A20FFF798FC5A4631462846FDF7CA
:1086280055FE1824009B494613F4000218BF012286
:108638004046FDF74BFE012239465046FDF746FEFF
:108648000A20FFF781FC002239465046FDF73EFE1E
:10865800009B013C4FEA430323F07F430093E1D1A1
:10866800012231462846FDF731FE0A20FFF76CFC4F
:10867800224631462846FDF729FE1824019B494623
:1086880013F4000218BF01224046FDF71FFE012225
:1086980039465046FDF71AFE0A20FFF755FC00221E
:1086A80039465046FDF712FE019B013C4FEA430351
:1086B80023F07F430193E1D1314601222846FDF79B
:1086C80005FE0A20FFF740FC22463146284603B043
:1086D800BDE8F04F04B0FDF7F9BD00000E4B82B0C5
:1086E8009A6942F001029A619A6902F001020092C5
:1086F800009ADA6942F08052DA61DB69074A03F0CE
:1087080080530193019B536823F0E06343F00073A7
:10871800536002B0704700BF0010024000000140E3
:10872800102230B5054689B00DEB0200002100F09B
:10873800F0FF2A682C4B9A4253D103F56C439A698F
:10874800032442F400729A619A6904A902F400723F
:108758000092009A9A69254842F010029A619A6933
:1087680002F010020192019A9A6942F004029A6199
:108778009A6902F004020292029A9A6942F0080287
:108788009A619B69059403F008030393039B0F23E5
:108798000493FDF7A9FCFF2304A915480493059445
:1087A800FDF7A2FC134804A904940594FDF79CFC6A
:1087B8008022114C114BE2604FF4007222614FF499
:1087C8000062236062610023202220466360A36068
:1087D800A261E361FDF79AF908B1FFF771FE2C6217
:1087E800656209B030BD00BF00240140001001409F
:1087F80000080140000C014040070020080002402A
:108808000268084B82B09A420AD103F50033DA694C
:1088180042F01002DA61DB6903F010030193019B57
:1088280002B070470010004070B5064686B01022AE
:10883800002102A800F06DFF32682B4B9A4251D1FB
:1088480003F558439A6902A942F480429A619A69E9
:10885800264802F480420092009A9A69002542F064
:1088680004029A619B69224C03F004030193019B63
:108878004FF4007302930223039303230593FDF738
:1088880033FC4FF48063194802A9029303950495B9
:10889800FDF72AFC174B204684E828008023A560B2
:1088A800E36025616561A561E561FDF72FF908B110
:1088B800FFF706FE4FF0100C0F4B746366620F4C07
:1088C800802284E8081000232046A360E260236128
:1088D8006361A361E361FDF719F908B1FFF7F0FDE2
:1088E8003463666206B070BD00380140000801407C
:1088F800BC06002058000240440002404806002000
:108908007047FEE7FEE7FEE7FEE7704770477047EF
:10891800FCF7D6BD0148FDF7E5B900BF40070020C8
:108928000148FDF7DFB900BF480600200148FDF700
:10893800D9B900BFBC0600200148FEF71BBC00BF28
:10894800000700200148FEF763B800BF8407002035
:1089580070B50E4615460C46A31B9D4201DC284601
:1089680070BDAFF3008004F8010BF5E708B50A4BBA
:108978000246196809B90949196069461868024424
:108988008A4206D900F090FE0C2303604FF0FF30B6
:1089980008BD1A6008BD00BF60040020E41700206D
:1089A8004FF0FF3070474FF4005300204B60704782
:1089B80001207047002070470E4B1A6842F00102F0
:1089C8001A6059680C4A0A405A601A6822F0847280
:1089D80022F480321A601A6822F480221A605A68D7
:1089E80022F4FE025A604FF41F029A60034A044BB5
:1089F8009A607047001002400000FFF8004000082D
:108A080000ED00E00B4B10B51B6804460021986888
:108A180001F064FB0023084A63602360A3600749F0
:108A2800A2F800340648A2F80234BDE8104001223A
:108A3800FEF7B2BA4C020020D00F0020D00B002065
:108A480000070020144A38B51068431C1360134B04
:108A5800596803F10C040D5D114C0131B1F5806FBB
:108A680025541446A8BF00229D68B8BF596005F177
:108A7800FF35A8BF5A609D606DB9094800F0A0FD98
:108A880022682946064800F044FE25600120BDE81A
:108A98003840FCF727BD38BD64040020C40B002013
:108AA800C407002000230F4A10B513600E4C0F4A6C
:108AB800136022680132B2F5806FB8BF1346236095
:108AC800A3680133B3F5806FA36001DBFFF7BAFF3A
:108AD800236807490122BDE8104019440548FEF7FC
:108AE8005BBA00BF5C040020C40B002050040020C7
:108AF800D00B00200007002008B5C3788178C25C3D
:108B08000130FEF772FD003018BF012008BD0000DB
:108B1800BE2310B50B4C60212370022363706123C0
:108B2800601CA170E370FEF745FDEB2384F861003B
:108B380084F862302146BDE8104063220248FEF7FF
:108B4800F1B900BFE305002000070020BE2310B5DF
:108B58000A4C032123700423601C6370A170E37026
:108B6800FEF728FDEB23A278207163712146BDE84A
:108B7800104003320248FEF7D5B900BF6804002050
:108B880000070020F0B5B54D02792B79A9B09342C2
:108B980004460CD0B24B029203F1100292E8030093
:108BA8008DE803000FCBFEF70DFC23792B7162795A
:108BB8006B7993420CD0AB4B029203F1100292E80E
:108BC80003008DE803000FCBFEF7FCFB63796B71A4
:108BD800A279AB7993420CD0A34B029203F1100215
:108BE80092E803008DE803000FCBFEF7EBFBA379B7
:108BF800AB71E279EB7993420CD09C4B029203F172
:108C0800100292E803008DE803000FCBFEF7DAFBB1
:108C1800E379EB71227A2B7A93420CD0944B02922F
:108C280003F1100292E803008DE803000FCBFEF772
:108C3800C9FB237A2B72627A6B7A93420CD08D4BE4
:108C4800029203F1100292E803008DE803000FCBB3
:108C5800FEF7B8FB637A6B72A27AAB7A93420CD0B8
:108C6800854B029203F1100292E803008DE803009D
:108C78000FCBFEF7A7FBA37AAB72E27AEB7A9342AB
:108C88000CD07E4B029203F1100292E803008DE8AB
:108C980003000FCBFEF796FBE37AEB72227B2B7B6C
:108CA80093420CD0764B029203F1100292E8030033
:108CB8008DE803000FCBFEF785FB237B2B73627BCC
:108CC8006B7B93420CD06F4B029203F1100292E837
:108CD80003008DE803000FCBFEF774FB637B6B7317
:108CE800A27BAB7B93420CD0674B029203F110023C
:108CF80092E803008DE803000FCBFEF763FBA37B2C
:108D0800AB73E27BEB7B93420CD0604B029203F196
:108D1800100292E803008DE803000FCBFEF752FB28
:108D2800E37BEB73237C2A7C9A4213D1697C627CB7
:108D380091420FD1A97CA27C91420BD1E97CE27CC3
:108D4800914207D1297D227D914203D1697D627DBF
:108D5800914220D04E4E2B743376637C98226B74EC
:108D680086F83430A37C06F11001AB7486F85030D5
:108D7800E37C6846EB7486F86C30237D2B7586F8A7
:108D88008830637D6B7586F8A43000F0B7FC96E8F0
:108D98000F00FEF759FCA37DAA7D9A4203D1E97D15
:108DA800E27D914235D0AB75E37DEB75A07DE37D27
:108DB80043EA002337485843FFF7CCFB364A374B82
:108DC80004924FF482620390029203F1100292E837
:108DD80003008DE803000FCBFFF7D0FB0120FCF761
:108DE80081FB22791E4B029203F1100292E80300E4
:108DF8008DE803000FCBFEF7E5FA1A4B6279029271
:108E080003F1100292E803008DE803000FCBFEF790
:108E1800D9FA237E2A7E607E9A4202D16A7E8242F5
:108E280070D02B76687640EA03201A4B5843FFF738
:108E380091FB194A1A4B04924FF4826203900292F2
:108E480003F1100292E803008DE803000FCBFFF74F
:108E580095FB0120FCF746FB24E000BFE30500205A
:108E680008000020200000203800002050000020CA
:108E7800680000208000002098000020B00000203A
:108E8800C8000020E0000020F800002010010020A9
:108E9800D8040020A086010092809F00B80100201D
:108EA800D0010020A279C54B029203F1100292E88A
:108EB80003008DE803000FCBFEF784FAE279C04B7C
:108EC800029203F1100292E803008DE803000FCB31
:108ED800FEF778FA227ABB4B029203F1100292E86D
:108EE80003008DE803000FCBFEF76CFAB64B627AED
:108EF800029203F1100292E803008DE803000FCB01
:108F0800FEF760FAA37EAA7EE07E9A4202D1EA7E4C
:108F1800824232D0AB76E87640EA0320AB4B584326
:108F2800FFF718FBAA4AAB4B04924FF482620390F6
:108F3800029203F1100292E803008DE803000FCBC0
:108F4800FFF71CFB0120FCF7CDFAA27AA24B029294
:108F580003F1100292E803008DE803000FCBFEF73F
:108F680031FA9E4BE27A029203F1100292E8030072
:108F78008DE803000FCBFEF725FA237F2A7F9A425C
:108F880003D1697F627F91424DD02B77637F6B77E6
:108F9800207F637F43EA00238C485843FFF7DAFABF
:108FA8008B4A8F4B04924FF482620390029203F132
:108FB800100292E803008DE803000FCBFFF7DEFAFA
:108FC8000120FCF78FFA227B864B029203F11002F4
:108FD80092E803008DE803000FCBFEF7F3F9627BFC
:108FE800814B029203F1100292E803008DE803001E
:108FF8000FCBFEF7E7F9A27B7C4B029203F110023C
:1090080092E803008DE803000FCBFEF7DBF9784BFD
:10901800E27B029203F1100292E803008DE803005C
:109028000FCBFEF7CFF9A37FAA7F9A4209D1E97F38
:10903800E27F914205D195F8201094F820209142C2
:1090480031D0AB77E37F0021EB7794F82030694883
:1090580085F82030E37FA27F1B0243EA024394F89D
:109068002020CDE90001134341F288320392022205
:10907800029242F2107226A85A430023FEF73CFCE3
:109088000322059241F2C2320492269A5A4B039265
:10909800279A029203F1100292E803008DE8030078
:1090A8000FCBFEF7B7FC94F8213095F821209A42AF
:1090B8000BD195F8221094F82220914205D195F809
:1090C800231094F82320914236D085F8213094F863
:1090D8002230002185F8223094F82330454885F85D
:1090E800233094F8223094F821201B0243EA0243EB
:1090F80094F82320CDE90001134341F2883203920A
:109108000222029242F2107226A85A430023FEF766
:10911800F3FB0322059241F2C2320492269A374B9E
:109128000392279A029203F1100292E803008DE855
:1091380003000FCBFEF76EFC94F8431095F843300C
:109148008B4206D04320FEF703FE94F8433085F89F
:10915800433094F8441095F844308B4206D04420AC
:10916800FEF7F6FD94F8443085F8443094F845103D
:1091780095F845308B4206D04520FEF7E9FD94F876
:10918800453085F8453094F8461095F846308B42BE
:1091980006D04620FEF7DCFD94F8463085F84630C8
:1091A80094F84A1095F84A308B4229D04A20FEF7A5
:1091B800CFFD94F84A3085F84A3021E03800002085
:1091C800500000206800002080000020A0860100D8
:1091D80092809F00E801002098000020B000002045
:1091E80000020020C8000020E0000020F800002055
:1091F80010010020005A6202340200201C020020E4
:1092080094F8491095F849308B4206D04920FEF76A
:109218009FFD94F8493085F8493094F8471095F83F
:1092280047308B4200F0BB8101264720FEF790FDB6
:1092380094F8473085F8473094F8481095F8483046
:109248008B4207D001264820FEF782FD94F848306B
:1092580085F8483094F84B1095F84B308B4245D040
:109268004B20FEF775FD94F84B30012085F84B3004
:10927800FCF738F994F84B30002B37D095F82230AA
:1092880095F821201B0243EA024395F82320002188
:10929800134341F2883203920222029242F2107280
:1092A800C2485A43CDE90001002326A8FEF724FB53
:1092B8000322059241F2C2320492269ABC4B0392D1
:1092C800279ABC4F029203F1100292E803008DE83E
:1092D80003000FCBFEF79EFB982207F110016846AA
:1092E80000F00CFA97E80F00FEF7AEF994F84C106E
:1092F80095F84C308B4243D04C20FEF729FD94F86A
:109308004C30012085F84C30FCF7ECF894F84C30E0
:10931800002B35D0EB7FAA7F1B0243EA024395F866
:1093280020200021134341F2883203920222029244
:1093380042F210729D485A43CDE90001002326A845
:10934800FEF7DAFA0322059241F2C2320492269A13
:10935800994B0392279A974F029203F1100292E8D1
:1093680003008DE803000FCBFEF754FB982207F1AA
:109378001001684600F0C2F997E80F00FEF764F99B
:1093880094F84D3095F84D209A4206D085F84D3026
:1093980094F84D104D20FEF7DBFC94F84E3095F80C
:1093A8004E209A4206D085F84E3094F84E104E2042
:1093B800FEF7CEFC814D94F84F3095F84F209A4235
:1093C80006D085F84F3094F84F104F20FEF7C0FCB8
:1093D80094F8503095F850209A4206D085F85030CD
:1093E80094F850105020FEF7B3FC94F8513095F8DB
:1093F80051209A4205D195F8521094F85220914282
:1094080006D0012685F8513094F8523085F852304C
:1094180094F8533095F853209A4205D195F8541092
:1094280094F85420914206D0012685F8533094F8D8
:10943800543085F8543094F8553095F855209A42B0
:1094480005D195F8561094F85620914206D0012679
:1094580085F8553094F8563085F8563094F85730DA
:1094680095F857209A4205D195F8581094F8582045
:10947800914206D0012685F8573094F8583085F87F
:10948800583094F8593095F859209A4205D195F8F2
:109498005A1094F85A20914206D0012685F859307E
:1094A80094F85A3085F85A3094F85B3095F85B2078
:1094B8009A4205D195F85C1094F85C20914206D048
:1094C800012685F85B3094F85C3085F85C3094F8B8
:1094D8005D3095F85D209A4205D195F85E1094F8B4
:1094E8005E20914206D0012685F85D3094F85E3002
:1094F80085F85E3094F85F3095F85F209A4205D180
:1095080095F8601094F8602091424AD085F85F3051
:1095180094F8603085F8603095F8523095F851002D
:1095280043EA0020FDF7CEFE95F8543095F8530035
:1095380043EA0020FDF7C6FE95F8563095F8550029
:1095480043EA0020FDF7BEFE95F8583095F857001D
:1095580043EA0020FDF7B6FE95F85A3095F8590011
:1095680043EA0020FDF7AEFE95F85C3095F85B0005
:1095780043EA0020FDF7A6FE95F85E3095F85D00F9
:1095880043EA0020FDF79EFE95F85F0095F86030ED
:1095980043EA002029B0BDE8F040FDF793BE00265D
:1095A8004AE6002EB8D129B0F0BD00BF005A6202C9
:1095B8001C020020D804002034020020E30500200B
:1095C80070B504464678FFF797FA054648B9A27879
:1095D80040F6B833033221461A48FDF747FC2846BF
:1095E80070BD032EFBD8DFE806F0022026290023F1
:1095F800154EA2785D1C0532DBB29A420FDA134889
:1096080000F064FDBFF34F8F1149124BCA6802F492
:10961800E0621343CB60BFF34F8F00BFFDE7E15C0F
:10962800304600F0DFFC2B46E3E72046FFF7AAFAB6
:10963800FFF78CFAD3E7FFF76BFAD0E70648FEF797
:109648001FFBF5E70007002057C000085DC00008B1
:1096580000ED00E00400FA05E3050020002103E026
:109668000B4B5B58435004310A480B4B42189A4243
:10967800F6D30A4A02E0002342F8043B084B9A4218
:10968800F9D3FFF799F900F015F8FEF71BFD7047BD
:1096980040C30008000000201C0400202004002013
:1096A800E4170020FEE70000014B1868704700BF70
:1096B8004C02002070B500250C4E0D4CA41BA410C4
:1096C800A54209D102F08AFC00250A4E0A4CA41BC7
:1096D800A410A54205D170BD56F82530984701352C
:1096E800EEE756F8253098470135F2E738C3000809
:1096F80038C3000838C300083CC3000810B5431E2F
:109708000A44914200D110BD11F8014B03F8014FF2
:10971800F7E703460244934200D1704703F8011B60
:10972800F9E7002B2DE9F0471E46BBBF03F10043C4
:109738001E4600232D2388B0149F129927F0200776
:10974800462F1446109DDDF84CA00B7004D0452F11
:1097580000D10135022300E0032307AA049206AAD8
:1097680003928DE828042246334600F0B9FE472FBD
:10977800804602D1119BDB0726D5462F08EB050949
:1097880011D198F80030302B0AD10022002320464E
:109798003146FBF779F918B9C5F10105CAF8005047
:1097A800DAF8003099440022002320463146FBF7BE
:1097B8006BF938B93022079B994505D9591C07918F
:1097C8001A70F8E7CDF81C904046079B159AA3EB52
:1097D8000803136008B0BDE8F0870346F7B5002911
:1097E80003F8022BB6BF2D222B22494209294270C9
:1097F80021DD0DF1070217460A2691FBF6F506FB57
:109808001511092D01F1300102F8011C02F1FF3494
:10981800294609DC3031023A04F8011CBA421C46D8
:1098280004D3201A03B0F0BD2246E6E712F8011B64
:1098380003F8011BF2E730221C46114404F8022BFE
:109848005970EEE72DE9F04F91B00C461A9F9346F8
:109858001E46054601F094FD036818460993FAF779
:10986800DFFC00230E933B680A90073323F00703BD
:1098780003F1080294F81880D4F800A03A60D3E9FC
:109888000023C4E91223D4F84C90A76C29F00043B4
:109898000B934FF0FF32A64B38460B99FBF726F98E
:1098A800002840F0F7814FF0FF32A14B38460B9962
:1098B800FBF7FEF8002840F0ED810022002338462F
:1098C8004946FBF7EBF810B12D2384F84330994B48
:1098D800994FB8F1470F98BF1F4603234FF000096F
:1098E80023612AF00403236000965B460FAA2146F1
:1098F800284600F0DFF9013040F09A804FF0FF3041
:1099080011B0BDE8F08F62680EA8531C0DF1340E3B
:109918004AF4806341D106226260002123600193EA
:1099280063680DF133020590029200933A464B4664
:109938000691CDF81080CDF80CE02846FFF7F1FE2F
:1099480008F0DF03472B074609D10D9BD81C02DB23
:109958006268934259DDA8F102085FFA88F8B8F105
:10996800650F0D9936D80139424604F150000D9122
:10997800FFF733FF0E9A81468318012A236102DC20
:109988002268D10701D5013323619DF83330002BBC
:10999800AAD02D2384F84330A6E7B8F1670F02D088
:1099A800B8F1470FB9D19AB1002106910DF13301F1
:1099B8008DE80C00236005903A46CDF81080CDF86C
:1099C8000CE002914B462846FFF7ABFE0746BCE782
:1099D8000122A1E7B8F1660F19D1002963680CDDEF
:1099E800216113B92268D20702D501330B442361E0
:1099F8000D9B4FF00009A365C7E713B92268D0078C
:109A080001D50233F3E70123F1E74FF067080D9B17
:109A18000E9A934205DB22682361D107E8D501330A
:109A2800E5E7002BCCBF0123C3F102031344DEE7B3
:109A380023685A0507D423693A4659462846B04749
:109A480001302AD15AE7B8F1650F40F2DC80D4E939
:109A5800120100220023FBF717F8002839D0012350
:109A6800364A59462846B04701303FF447AF0E9B67
:109A78000D9A9A4202DB2368D8070ED50A9B099AE9
:109A880059462846B04701303FF438AF002704F163
:109A98001A080E9B013B9F4211DB23689F0708D5DC
:109AA800002704F11908E3680F9A9B1A9F42C0F235
:109AB800E780E0680F9B9842B8BF184620E701236B
:109AC800424659462846B04701303FF417AF0137A0
:109AD800DFE70D9B002B33DC0123184A5946284643
:109AE800B04701303FF40AAF0D9B23B90E9B13B961
:109AF8002368D907D1D50A9B099A59462846B04701
:109B080001303FF4FBAE4FF0000804F11A090D9B39
:109B18005B42984501DB0E9B8EE701234A46594676
:109B28002846B04701303FF4E9AE08F10108EEE7F6
:109B3800FFFFEF7F70C0000874C0000880C00008F5
:109B48000E9AA36D9A42A8BF1A46002A904636DCA0
:109B58004FF0000A04F11A0328EAE8780B93D4F8C6
:109B68005890A9EB08039A4531DB0E9B0D9A9A424F
:109B780038DB2368DA0735D40E9B0D99A3EB09026D
:109B8800A3EB01089045A8BF9046B8F1000F31DC5F
:109B9800002728EAE87804F11A090D9A0E9B9B1A07
:109BA800A3EB08039F42BFF678AF01234A46594604
:109BB8002846B04701303FF4A1AE0137EDE7134620
:109BC80059463A462846B0470130C1D196E60123A6
:109BD8000B9A59462846B04701303FF48FAE0AF138
:109BE800010ABCE70A9B099A59462846B047013042
:109BF800C2D183E6434607EB090259462846B047D7
:109C08000130C5D17AE60E9A012A01DCDB0734D58A
:109C180001233A4659462846B04701303FF46EAE14
:109C28000A9B099A59462846B04701303FF466AE68
:109C3800D4E9120100220023FAF726FF50B10027C9
:109C480004F11A080E9B013B9F420CDB4B4604F1C2
:109C58005002F2E60E9B7A1C013B59462846B04753
:109C68000130F3D14AE60123424659462846B04717
:109C780001303FF443AE0137E4E701233A46ECE70D
:109C88000123424659462846B04701303FF436AED4
:109C9800013708E73A464B4638464946FAF726FF61
:109CA80000283FF430AE014B014F12E678C000089F
:109CB8007CC000082DE9F04791461F468A680B6969
:109CC80006469342B8BF1346C9F8003091F84320BE
:109CD8000C46DDF8208012B10133C9F80030236842
:109CE800990642BFD9F800300233C9F80030256818
:109CF80015F0060507D104F1190AE368D9F8002020
:109D08009B1A9D422ADB94F843302268003318BF1F
:109D1800012392062FD404F1430239463046C04746
:109D2800013022D02368E56803F00603042B18BF2E
:109D38000025D9F800204FF0000908BFAD1AA36824
:109D4800226908BF25EAE5759342C4BF9B1AED183E
:109D58001A344D451BD10020BDE8F0870123524637
:109D680039463046C047013003D14FF0FF30BDE8D7
:109D7800F0870135C1E73020E11881F843005A1C0B
:109D880094F845102244023382F84310C3E70123B4
:109D9800224639463046C0470130E6D009F101096C
:109DA800D7E700002DE9F04317460A7E85B06E2AF2
:109DB800984606460C460C9B01F1430E00F0BC8009
:109DC8001AD8632A2ED00AD8002A00F0C880582A48
:109DD80000F08A8004F1420584F842202AE0642ACF
:109DE80001D0692AF6D121681A6811F0800F23D0B2
:109DF800111D1960136827E0732A00F0B48008D891
:109E08006F2A2AD0702AE5D10A6842F020020A6037
:109E180003E0752A21D0782ADCD178226F4984F8AA
:109E2800452064E01A6801F14205111D19601368A4
:109E380084F842300123A3E011F0400F02F104013D
:109E48001960D7D0B2F90030002B03DA2D225B421B
:109E580084F8432062490A2217E02068196810F044
:109E6800800F03D0081D18600B6806E010F0400F43
:109E780001F104001860F7D00B886F2A14BF0A227A
:109E880008225749002084F843006568002DA56022
:109E9800C0F29C80206820F004002060002B3FD195
:109EA800002D40F095807546082A0BD12368DA0703
:109EB80008D5236962689A42DEBF302305F8013C61
:109EC80005F1FF35AEEB05032361CDF800803B4675
:109ED80003AA21463046FFF7EDFE013055D14FF079
:109EE800FF3005B0BDE8F08381F845203C49226881
:109EF800186812F0800F00F104051D6001D0036896
:109F080002E05506FBD50388D00744BF42F0200283
:109F180022601BB9226822F0200222601022B1E7D9
:109F28007546B3FBF2F002FB1033CB5C05F8013D3C
:109F380003460028F5D1B7E708681A6810F0800FC3
:109F4800496904D0101D18601368196007E010F003
:109F5800400F02F1040018601368F6D0198000233E
:109F680075462361B1E71A68111D1960156800214B
:109F78006268284601F07EFA08B1401B6060636899
:109F88002361002384F843309FE723692A46394632
:109F98003046C0470130A2D023689B0707D500256B
:109FA80004F11909E368039A9B1A9D4205DBE068EE
:109FB800039B9842B8BF184693E701234A4639469F
:109FC8003046C04701308AD00135EBE7002BA7D1D6
:109FD8000B7804F1420584F8423065E793C0000825
:109FE80082C000080FB40A4B13B51C6824B1A369DA
:109FF80013B9204601F03AF905AB049AA168204646
:10A00800019301F0F7FD02B0BDE8104004B07047BD
:10A018004C02002070B50E46054618B183690BB98D
:10A0280001F024F9AB69AC6813B9284601F01EF9B0
:10A03800234B9C4217D16C68A3891B071DD5236944
:10A04800DBB1013EA36816F8011F013BA360E9B923
:10A05800002B2EDA22460A21284600F0F5F80130B6
:10A0680011D00A2070BD174B9C4201D1AC68E3E7C0
:10A07800154B9C4208BFEC68DEE72146284600F0F5
:10A0880035F90028DDD04FF0FF3070BD002B04DA21
:10A09800A269934206DB0A2904D023685A1C22606D
:10A0A8001970CFE72246284600F0CEF80130C9D112
:10A0B800E9E70A2023685A1C2260187070BD00BFA7
:10A0C800D4C00008F4C00008B4C00008024B014620
:10A0D8001868FFF79FBF00BF4C02002000294FF40B
:10A0E80080630CBF0222002200F000B82DE9F7437C
:10A0F8001D46514B04461E680F46904626B1B3696B
:10A1080013B9304601F0B2F84C4B9C4252D17468F6
:10A11800B8F1020F06D0B8F1010F00F28980002DC6
:10A12800C0F286802146304601F036F8616B41B1B5
:10A1380004F14403994202D0304601F089FC00231F
:10A1480063630023A3616360A3891B0603D52169A8
:10A15800304601F07DFCA389B8F1020F23F44A636D
:10A1680023F00303A3815DD001AB6A462146304644
:10A1780001F014F9A3891843A0812DBB009D28463E
:10A1880001F070F9074600284ED1DDF80090A94586
:10A198003CD14FF0FF30A38943F00203A381002391
:10A1A800A36004F14703236023610123636103B0C3
:10A1B800BDE8F083224B9C4201D1B468A8E7214B4B
:10A1C8009C4208BFF468A3E7002FD8D0B36913B93D
:10A1D800304601F04BF8B8F1010F08BFA38927609A
:10A1E80004BF43F00103A381A389276113F008008A
:10A1F80065611BD013F001004FF000031FBF6D42D3
:10A20800A360A561184608BFA560D0E7484601F0DD
:10A2180029F907460028BCD0A3894D4643F080039E
:10A22800A381D3E70020B6E7A946F5E7A060BEE71B
:10A238004FF0FF30BBE700BF4C020020D4C000083D
:10A24800F4C00008B4C00008F8B50E461446054628
:10A2580018B183690BB901F009F8214B9C422AD146
:10A268006C68A369A360A3891A072ED5236963B311
:10A2780023692068F6B2C01A63693746984204DB3E
:10A288002146284600F088FF28BBA3680130013B1F
:10A29800A36023685A1C22601E706369984204D028
:10A2A800A389DB0719D50A2E17D12146284600F0C5
:10A2B80073FF90B10FE00B4B9C4201D1AC68D0E723
:10A2C800094B9C4208BFEC68CBE72146284600F0C2
:10A2D8000DF80028CCD04FF0FF373846F8BD00BF46
:10A2E800D4C00008F4C00008B4C00008324B70B5F0
:10A2F8001D6806460C4625B1AB6913B9284600F01F
:10A30800B5FF2E4B9C420FD16C68B4F90C309AB251
:10A3180015072CD4D00611D40922326043F040032B
:10A32800A3814FF0FF3070BD254B9C4201D1AC6832
:10A33800EBE7244B9C4208BFEC68E6E7510712D5CF
:10A34800616B41B104F14403994202D0304601F0F7
:10A358007FFB00236363A38923F02403A3810023E5
:10A36800636023692360A38943F00803A3812369F9
:10A378004BB9A38903F42073B3F5007F03D02146BA
:10A38800304601F02FF8A28912F001030CD0002307
:10A39800A36063695B42A361236953B9B4F90C30C4
:10A3A80013F08000BAD170BD920758BF6369A360EB
:10A3B800F2E70020F7E700BF4C020020D4C00008F5
:10A3C800F4C00008B4C000082DE9F74F03690C6910
:10A3D80080469C4200F38280013C01F1140700F1A1
:10A3E800140657F8245056F824000135B0FBF5F54B
:10A3F8004FEA840E06EB0E0307EB0E0901938DB3AB
:10A408004FF0000A3846B446D34650F8042B93B2AE
:10A4180005FB03A3120C4FEA134A05FB02A29BB2E9
:10A42800ABEB0303BCF800B04FEA124A5B441FFAD7
:10A4380082FBDCF800208145CBEB124202EB234281
:10A448009BB243EA02434FEA224B4CF8043BDCD26E
:10A4580056F80E3033B9019B043B9E421A4631D35D
:10A46800C8F81040404601F01CFA002826DB3046A8
:10A478004FF0000E013557F8041BD0F800C08BB21E
:10A48800AEEB03031FFA8CF213440A0CC2EB1C4216
:10A4980002EB23429BB243EA0243B9454FEA224EFC
:10A4A80040F8043BE7D256F8242006EB84032AB987
:10A4B800043B9E421A460BD3C8F81040284603B006
:10A4C800BDE8F08F1268043B002AC9D1013CC4E7FB
:10A4D8001268043B002AEFD1013CEAE70020EEE7CE
:10A4E8002DE9F04F466A95B00446219DCDE9022337
:10A4F8003EB9102000F0B6FF6062466086600660D4
:10A50800C660636A196851B15A68012393404A606A
:10A518008B60204600F0F0FF0022636A1A60039BFC
:10A52800002BB7BF012300232B60039BAEBF2B601A
:10A5380023F000430393DDF80C90AB4B33EA090397
:10A548001BD142F20F73209A1360029B23B9C9F3FF
:10A558001300002800F08385229B53B9A34B21E008
:10A56800A34B06930833229A1360069815B0BDE8EA
:10A57800F08F9E4B06930333F5E7DDE9026700226F
:10A58800002330463946FAF77FFA804660B1012346
:10A59800209A1360229B002B00F05E85954B229A2F
:10A5A8001360013B0693E0E712AB019313AB0093F2
:10A5B80032463B46204601F0EDF9C9F30A5582467A
:10A5C800002D7DD03046C7F3130343F07F5141F48B
:10A5D8004011A5F2FF35CDF840800022864BF9F7EF
:10A5E80037FE7BA3D3E90023F9F7E6FF7AA3D3E983
:10A5F8000023F9F72FFE064628460F46F9F776FF9F
:10A6080077A3D3E90023F9F7D7FF02460B46304674
:10A618003946F9F71FFE06460F46FAF77DFA00227B
:10A628008346002330463946FAF738FA58B1584677
:10A63800F9F75CFF02460B4630463946FAF724FA2A
:10A6480008B90BF1FF3BBBF1160F58D8DDE902231F
:10A658006A4901EBCB01D1E90001FAF73DFA00287C
:10A668004FD000230BF1FF3B0D93129B5D1B6B1E1C
:10A67800079343BF0023C5F1010807934FF0000873
:10A68800BBF1000F3FDB079BCDF830B05B4407936D
:10A69800002308931E9B092B00F2B480052BC4BF2E
:10A6A800043B1E931E9BC8BF0026A3F10203D8BF1C
:10A6B8000126032B00F2B280DFE803F084862D78B0
:10A6C800139B129D1D4405F23243202B11DD029A83
:10A6D80005F21240C3F1400322FA00F009FA03F32D
:10A6E8001843F9F7F3FE0123A1F1F871013D109326
:10A6F80073E7C3F12000029B03FA00F0F1E701239E
:10A70800B2E70D90B1E7CBF1000308930023A8EB63
:10A718000B080C93BEE7012309931F9B002B40F302
:10A7280080809946049300220421656A6A6001F1D9
:10A7380014029A427AD96968204600F0A9FE636A31
:10A7480028601B68B9F10E0F069300F2F080002E06
:10A7580000F0ED80DDE90223BBF1000FCDE90E2307
:10A7680079DD264A0BF00F034FEA2B1602EBC303E1
:10A77800F006D3E90023CDE90A235CD5DDE90E0113
:10A788001F4B0325D3E90823FAF740F8CDE9020166
:10A7980006F00F061A4F002E4FD1DDE90A23DDE936
:10A7A8000201FAF733F8CDE902016EE001230993BB
:10A7B8001F9B5B4403F1010904934B46012BB8BF6F
:10A7C8000123B0E70023A7E70023F0E7AFF30080F9
:10A7D80061436F63A787D23FB3C8608B288AC63F9F
:10A7E800FB799F501344D33F0000F07FADC00008B1
:10A7F800A4C0000881C000080000F83F40C100085C
:10A8080018C100080126002309961E934FF0FF3354
:10A8180000220493994612231F9284E70123099387
:10A82800F4E70123049399461A46F5E76A68490054
:10A8380001326A607BE70225ACE7F10708D5DDE95C
:10A848000A01D7E90023F9F7B7FECDE90A01013576
:10A85800761008379FE700F0A580DDE90E01CBF1FF
:10A868000006A24B06F00F0203EBC203D3E9002354
:10A87800F9F7A2FE02250023CDE902019C4F36110B
:10A88800002E40F08480002B8DD10D9B002B00F012
:10A898008B80DDE90223CDE90A23DDE90A010022E4
:10A8A800944BFAF7FBF800287ED0B9F1000F7BD063
:10A8B800049B002B37DDDDE90A0100228E4BF9F7F6
:10A8C8007BFECDE90201049E0BF1FF3701352846D6
:10A8D800F9F70CFEDDE90223F9F76EFE874B00223B
:10A8E800F9F7B8FCCDE90A010B9BA3F150750B955C
:10A8F800002E5CD1DDE902010022814BF9F7A8FCAA
:10A908000A9A2B46CDE90201FAF7E6F8002840F04A
:10A91800F782DDE902010A9A05F10043FAF7BEF869
:10A92800002840F0EB82DDE90E23CDE90223139BDA
:10A93800002BC0F25081BBF10E0F00F34C816B4B22
:10A9480003EBCB03D3E90023CDE904231F9B002BA2
:10A9580080F2DA80B9F1000F00F3D68040F0CD82A2
:10A96800DDE904010022664BF9F726FEDDE9022342
:10A97800FAF7A8F84E464F46002840F0A482069BF6
:10A98800069A5D1C31230BF1010B13709FE2F2074D
:10A9980005D5D7E90023F9F70FFE01230135761015
:10A9A80008376DE7022570E75F464E468FE7069A3F
:10A9B8004E4B32441192099A711E002A48D003EB7B
:10A9C800C103D3E9002300204E49F9F71FFFDDE951
:10A9D8000A23F9F73DFCCDE90A01069DDDE90201EC
:10A9E800FAF79AF80646F9F781FD02460B46DDE9C3
:10A9F8000201F9F72DFCDDE90A23303605F8016B71
:10AA0800CDE90201FAF74AF8002864D1DDE902230A
:10AA180000203849F9F71CFCDDE90A23FAF73EF86B
:10AA2800002840F0B980119B9D423FF47CAFDDE9DE
:10AA38000A010022304BF9F7BFFD0022CDE90A01D7
:10AA4800DDE902012C4BF9F7B7FDCDE90201C5E7B5
:10AA580003EBC101D1E90001DDE90A23F9F7ACFDF7
:10AA6800CDE90A01069DDDE90201FAF755F8064627
:10AA7800F9F73CFD02460B46DDE90201F9F7E8FB70
:10AA88003036119B05F8016BAB42CDE902014FF05E
:10AA9800000224D11B4BDDE90A01F9F7DBFB024672
:10AAA8000B46DDE90201FAF717F8002874D1DDE951
:10AAB8000A2300201349F9F7CBFB02460B46DDE9D0
:10AAC8000201F9F7EBFF00283FF42DAF15F8013C20
:10AAD8006A1E302B01D0BB464DE01546F6E7064B03
:10AAE800F9F76AFDCDE90201BDE700BF40C10008E2
:10AAF80018C100080000F03F0000244000001C407E
:10AB0800000014400000E03F069DDDE90267DDE932
:10AB1800042330463946F9F779FEF9F7FDFF8046F8
:10AB2800F9F7E4FCDDE90423F9F746FD02460B4694
:10AB380030463946F9F78CFB08F1300605F8016B09
:10AB4800069E0246AE1BB1450B4637D1F9F782FB8C
:10AB580006460F4602460B46DDE90401F9F79EFF5B
:10AB6800C8B9DDE9040132463B46F9F78DFF10B15B
:10AB780018F0010F0FD15146204600F0BDFC00230C
:10AB8800209A2B700BF101031360229B002B3FF4DA
:10AB9800ECAC1D60E9E45F4615F8012C6B1E392A00
:10ABA80006D1069A9A4207D130231370134601370B
:10ABB8001A7801321A708EE71D46EDE70022B54B70
:10ABC800F9F7FAFC0022002306460F46F9F75CFF66
:10ABD80000289CD0CFE7099A002A00F029811E9A04
:10ABE800012A00F30E81109A002A00F0068103F270
:10ABF80033434546089E079A01211A442046984443
:10AC0800079200F019FD0746002D0BDD079B002B6E
:10AC180008DDAB42A8BF2B46079AA8EB0308ED1A3C
:10AC2800D31A0793089BFBB1099B002B00F0048102
:10AC3800002E11DD39463246204600F093FD52467B
:10AC480001460746204600F000FD51460A9020467E
:10AC580000F052FC0A9B9A46089B9A1B04D0514666
:10AC6800204600F07FFD82460121204600F0E4FCEA
:10AC78000C9B0646002B40F3E1801A46014620460D
:10AC880000F070FD1E9B0646012B40F3DA8000237E
:10AC98000893336906EB8303186900F07FFCC0F161
:10ACA8002000079B184410F01F0000F0F080C0F14E
:10ACB8002003042B40F3E280079BC0F11C00804472
:10ACC800054403440793B8F1000F05DD5146424699
:10ACD800204600F095FD8246079B002B05DD314696
:10ACE8001A46204600F08CFD06460D9B002B00F00E
:10ACF800D3803146504600F0D4FD002880F2CC8045
:10AD0800002351460A22204600F00DFC099B0BF156
:10AD1800FF3B8246002B00F0A981002339460A2216
:10AD2800204600F000FC049B0746002B03DC1E9B1A
:10AD3800022B00F3B980002D05DD39462A4620464E
:10AD480000F05EFD0746089B002B00F01081796833
:10AD5800204600F09DFB05463A6907F10C010232D6
:10AD680092000C30FEF7CAFC01222946204600F06A
:10AD780047FD07970746029BDDF8188003F001039B
:10AD8800089331465046FFF71FFB0799054600F127
:10AD98003009504600F085FD3A460290314620467B
:10ADA80000F099FDC3680246002B40F0E28001469E
:10ADB8000990504600F075FD0346099A1146204651
:10ADC800099300F099FB099B002B40F0D4801E9A50
:10ADD800002A40F0D080089A002A40F0CC80B9F1CF
:10ADE800390F00F0E880029B002B01DD05F13109E5
:10ADF80008F1010588F800906BE0129BC3F1360357
:10AE0800F7E6089B09F1FF36B342B7BF089B9E1BC4
:10AE1800F21A0C9BBFBF08969B180C930026B9F139
:10AE2800000FB9BFA8EB0905002345464B46E2E6EB
:10AE3800089E4546099FE7E6089A10E71E9B012BE6
:10AE480018DC029BB3B9039BC3F31303A3B9039B99
:10AE580023F000431B0D1B052BB1079B08F10108CC
:10AE680001330793012308930C9B002B7FF411AF48
:10AE7800012016E70023F6E7029BF4E73FF423AF2F
:10AE8800079A1C331A4498441D4413461AE703468C
:10AE9800F6E700BF00002440B9F1000F33DC1E9B29
:10AEA800022B30DDCDF81090049B63B931460522A2
:10AEB800204600F038FB01460646504600F0F1FCFB
:10AEC80000283FF75CAD1F9B069D6FEA030B00232C
:10AED80007933146204600F00FFB002F3FF44BAE9E
:10AEE800079B2BB1BB4203D01946204600F004FB58
:10AEF8003946204600F000FB3DE600263746E2E7EB
:10AF0800BB4637463BE5099BCDF81090002B7FF4F4
:10AF180012AF069D31465046FFF756FA069B00F1E0
:10AF2800300905F8019B049AEB1A9A4200F38180D4
:10AF3800069B012AACBF9B18013398460023079350
:10AF480051460122204600F05BFC3146824600F063
:10AF5800A8FC002834DC02D119F0010F30D1454695
:10AF680015F8013C6A1E302BB3D11546F8E7384670
:10AF7800FFE6012322E7029A002A04DB28D11E9A61
:10AF880032BB089A22BB002B7FF732AF5146012211
:10AF9800204600F035FC3146824600F082FC00284D
:10AFA80005DC7FF425AF19F0010F3FF421AFB9F1AB
:10AFB800390F7FF41BAF392308F1010808F8013C69
:10AFC800454615F8013C6A1E392B3AD001333FE05B
:10AFD800002B08F1010505DDB9F1390FEBD009F1B6
:10AFE800010907E7069B049AEB1A9342A84605F85D
:10AFF800019CA5D0514600230A22204600F093FA6E
:10B00800079B8246BB424FF00A024FF000030799A4
:10B01800204604D100F087FA07900746B1E600F011
:10B0280082FA002307900A223946204600F07BFA6C
:10B03800F3E7514600230A22204600F074FA8246BC
:10B0480068E7069B934205D13123069A0BF1010B61
:10B0580013703EE71546B4E7094BFFF7A3BA229BE6
:10B06800002B7FF47DAA074BFFF79CBA049B002BAB
:10B078003FF74FAF1E9B022B7FF74BAF14E700BF84
:10B0880080C00008A4C000088A892DE9F04105465F
:10B0980010070C465AD44B68002B05DC0B6C002BB0
:10B0A80002DC0020BDE8F081E66A002EF9D000231A
:10B0B80012F480522F682B6033D0606DA3895A0731
:10B0C80005D56368C01A636B0BB1236CC01A0023E3
:10B0D8000246E66A216A2846B047431CA38906D17E
:10B0E80029681D294BD82B4ACA40D60747D50022C4
:10B0F80062602269D904226004D5421C01D12B6800
:10B1080003B96065616B2F600029CAD004F144035C
:10B11800994202D0284600F09BFC00206063BDE8FD
:10B12800F081216A01232846B047411CC6D12B680B
:10B13800002BC3D01D2B01D0162B01D12F60B0E7F7
:10B14800A38943F04003A381BDE8F0810F69002F74
:10B15800A7D0930718BF00230E6808BF4B69A6EB5A
:10B1680007080F608B60B8F1000F9ADD43463A4636
:10B17800216A2846A66AB047002807DCA38943F05D
:10B188004003A3814FF0FF30BDE8F0810744A8EBEE
:10B198000008E8E70100402038B50B6905460C4671
:10B1A800DBB118B183690BB900F060F80C4B9C4215
:10B1B80009D16C68B4F90C307BB121462846BDE84A
:10B1C8003840FFF761BF074B9C4201D1AC68F1E7FB
:10B1D800054B9C4208BFEC68ECE7002038BD00BF77
:10B1E800D4C00008F4C00008B4C00008014900F049
:10B1F800A9B800BFA1B10008002310B50446036038
:10B208004360836081814366C281036143618361D6
:10B21800194608225C30FEF77CFA054B246263620B
:10B22800044BA362044BE362044B236310BD00BFCD
:10B2380049BE00086BBE0008A3BE0008C7BE0008D0
:10B2480070B568254A1E55430E4605F1740100F095
:10B258004BFC044640B1002180E842000C30A0605D
:10B2680005F16802FEF755FA204670BD836910B5EE
:10B27800044633BB8364C3640365124B124A1B68DC
:10B288008262984204BF0123836100F01FF8606066
:10B29800204600F01BF8A060204600F017F80022B6
:10B2A800E06004216068FFF7A7FF01220921A06878
:10B2B800FFF7A2FF02221221E068FFF79DFF01239A
:10B2C800A36110BD6CC00008F5B10008F8B51C4BAF
:10B2D80007461E68B36913B93046FFF7C7FF4836FB
:10B2E800B4687368013B03D5336833B13668F7E750
:10B2F800B4F90C506DB16834F4E704213846FFF70F
:10B308009FFF30600028F1D10C2304463B602046A3
:10B31800F8BD4FF6FF73E38101236566A3812560BD
:10B32800A560656025616561A5610822294604F16B
:10B338005C00FEF7EEF96563A563A564E564E6E7DE
:10B348006CC000082DE9F84380468946002600F1C4
:10B35800480414B93046BDE8F883A5686768013F1A
:10B3680001D52468F5E7AB89012B07D9B5F90E306B
:10B37800013303D029464046C84706436835EEE7FF
:10B38800044B1B68186A044B002808BF1846F030A5
:10B39800704700BF4C020020B002002070B50E4676
:10B3A800B1F90E1090B0002914461D4607DA0023A3
:10B3B8002B60B3891A0610D44FF480630EE001AAFB
:10B3C80000F0A4FD0028F2DB029A02F47042A2F514
:10B3D80000535A425A412A60EEE740230020236076
:10B3E80010B070BD8B8973B59D0706460C4607D50E
:10B3F80004F14703236023610123636102B070BD38
:10B4080001AB6A46FFF7CAFF00990546304600F0CF
:10B418006BFB48B9B4F90C309A05EFD423F0030359
:10B4280043F00203A381E3E70D4BB362A3892060D5
:10B4380043F08003A381009B20616361019B5BB1A2
:10B44800B4F90E10304600F073FD28B1A38923F03B
:10B45800030343F00103A381A3891D43A581CDE71D
:10B46800F5B10008024B0146186800F03DBB00BF6B
:10B478004C02002010B5C9B202449042034601D1E3
:10B48800002010BD1C7801308C42F6D1184610BD42
:10B4980070B5456A04460E463DB91020FFF7E2FF35
:10B4A8006062456085600560C560656AEB6883B168
:10B4B800636ADB6853F82600B8B9012101FA06F57A
:10B4C8006A1D9200204600F0B4FA60B146608560BB
:10B4D8000EE021220421204600F0ABFA636AE860FE
:10B4E800DB68002BE4D1002070BD026843F82620F9
:10B4F80000230361C36070BD70B5446A06460D46FB
:10B508003CB91020FFF7AEFF7062446084600460AD
:10B51800C4603DB1736A6A68DB6853F82210296019
:10B5280043F8225070BD2DE9F0411F4606460C46EF
:10B5380000230D6901F1140EDEF80000013381B219
:10B5480002FB0171000C0F0C02FB007089B201EBC9
:10B5580000419D424FEA10474EF8041BECDCD7B17E
:10B56800A3689D4212DB616830460131FFF790FF06
:10B578008046226904F10C01023292000C30FEF779
:10B58800BDF821463046FFF7B7FF444604EB850374
:10B5980001355F6125612046BDE8F081020C120487
:10B5A8000346B2B90304102013F07F4F04BF1B02F7
:10B5B800083013F0704F04BF1B01043013F0404FE4
:10B5C80004BF9B000230002B06DB5B0003D5013073
:10B5D80070470020E8E7202070470368014613F011
:10B5E80007020BD0DA0723D4980749BF5B089B08EA
:10B5F80001200B605CBF0B600220704798B2A8B9AD
:10B6080010201B0C13F0FF0F04BF1B0A08301A0789
:10B6180004BF1B0904309A0704BF9B080230DA07ED
:10B6280002D45B0806D001300B6070471046E9E78A
:10B63800002070472020704710B50C460121FFF705
:10B6480027FF01224461026110BD2DE9F74F14461E
:10B658000A69236989469A42BEBF0B46A1461C4621
:10B66800D9F81070D4F810A0D9F80830D9F8041017
:10B6780007EB0A069E42C8BF0131FFF709FF00F138
:10B6880014052B46002205EB8608434516D304F122
:10B69800140209F1140102EB8A0301EB87070193F5
:10B6A800019C134694420CD8002E03DD58F8043D43
:10B6B800002B54D0066103B0BDE8F08F43F8042B8B
:10B6C800E3E7B3F800A00432BAF1000F20D0AE4689
:10B6D80089464FF0000C59F8044BBEF800B0A3B2ED
:10B6E8000AFB03B34FEA144BDEF8004063444FEA09
:10B6F800144C0AFB0BC404EB13449BB243EA044307
:10B708004F454FEA144C4EF8043BE4D8CEF800C03D
:10B7180032F8029CB9F1000F1FD0AE468C464FF0AC
:10B72800000A2B68BCF80040BEF802B09BB209FBC7
:10B7380004B4A24443EA0A434EF8043B5CF8043BD1
:10B74800BEF800401B0C09FB0343674503EB1A4393
:10B758004FEA134AE6D8CEF800300435A0E7013E98
:10B76800A2E700002DE9F843154612F00302064649
:10B778000F4607D0214C013A002354F82220FFF746
:10B78800D2FE0746AD1035D0746A3CB91020FFF7D9
:10B7980069FE7062446084600460C460D6F82480E6
:10B7A800D8F808404CB940F271213046FFF744FF01
:10B7B80000230446C8F8080003604FF00008EB07B0
:10B7C8000AD5394622463046FFF73FFF81463946BB
:10B7D8003046FFF791FE4F466D100BD0206838B900
:10B7E800224621463046FFF730FF2060C0F800802F
:10B7F8000446E4E73846BDE8F88300BF08C20008FD
:10B808002DE9F0470C460746164623694FEA621AA7
:10B818000AEB03094968A36809F10105AB4231DB6A
:10B828003846FFF735FE00228046114600F1140322
:10B8380052452ADB20692AEAEA7A04F1140116F053
:10B848001F0203EB8A0301EB800E22D00020C2F115
:10B85800200C0E689640304343F8040B51F8040B53
:10B868008E4520FA0CF0F4D8186008B109F10205E9
:10B87800013D3846C8F810502146FFF73DFE4046C6
:10B88800BDE8F08701315B00C8E743F822100132B8
:10B89800CEE7043B51F8042B8E4543F8042FF9D822
:10B8A800E6E703690A6930B59B1A0CD19200143097
:10B8B80014318418114454F8045D51F8042D95424C
:10B8C80003D005D30123184630BDA042F3D3FAE7CD
:10B8D8004FF0FF33F7E72DE9F0470D4607461146CD
:10B8E80028461446FFF7DDFF061E08D131463846C4
:10B8F800FFF7CEFD012346610361BDE8F087A4BFD1
:10B9080023462C4638466168A6BF1D4600260126F8
:10B91800FFF7BEFD4FF0000CC6602B69266904F1E5
:10B92800140205F1140902EB860709EB830800F1FC
:10B93800140152F804AB59F8045B1FFA8AF3634404
:10B94800ACB21B1B2C0CC4EB1A4404EB23449BB273
:10B958004FEA244CC84543EA0444964641F8044B50
:10B96800E7D8BE4505D351F8043D8BB10661BDE863
:10B97800F0875EF8044BA2B26244131403EB14433D
:10B9880092B242EA03424FEA234C41F8042BE8E71B
:10B99800013EE8E72DE9F3411C4601219046089E47
:10B9A800099DFFF775FDC4F31302C4F30A54074653
:10B9B80034BB0192B8F1000F27D002A840F8088DD7
:10B9C800FFF70BFE0099F0B1019AC0F1200302FACB
:10B9D80003F30B43C2407B610192019B002B14BF10
:10B9E80002210121BB613961C4B1A4F2334404448A
:10B9F8003460C0F135002860384602B0BDE8F081F7
:10BA080042F48012D5E77961E7E701A8FFF7E5FD81
:10BA18000121019B39617B612030E5E7A0F23240CA
:10BA280007EB810330601869FFF7B8FDC0EB4110E0
:10BA3800E1E738B502FB01F4214600F055F8054668
:10BA480018B122460021FDF764FE284638BD0000E3
:10BA580038B50546002943D051F8043C0C1F002B8B
:10BA6800B8BFE41800F098FA1E4A1368104633B9B4
:10BA7800636014602846BDE8384000F08EBAA342DF
:10BA88000BD921686218934201BF1A685B68521883
:10BA9800226063600460EDE713465A680AB1A24267
:10BAA800FAD919685818A0420BD1206801445818CF
:10BAB80082421960DED110685268014419605A60E8
:10BAC800D8E702D90C232B60D4E7206821188A42D2
:10BAD80001BF116852680918216062605C60C9E79B
:10BAE80038BD00BF7004002070B5CD1C25F00305DB
:10BAF80008350C2D38BF0C25002D064601DBA94260
:10BB080003D90C233360002070BD00F045FA234AA6
:10BB18001468214691B9224C23681BB9304600F0BD
:10BB28007FF920602946304600F07AF9431C26D177
:10BB38000C233046336000F030FAE4E70B685B1BF7
:10BB48001AD40B2B0FD90B60CC18CD50304600F00F
:10BB580024FA04F10B00231D20F00700C31A1BD0A0
:10BB68005A42E25070BD8C420BBF63684B68136049
:10BB7800636018BF0C46E9E70C464968CAE7C41C6D
:10BB880024F00304A04205D0211A304600F048F9F9
:10BB98000130CDD02560D9E770BD00BF700400200A
:10BBA80074040020936810B4013B002B936008DAFA
:10BBB8009469A34202DBCBB20A2B02D110BCFEF778
:10BBC80043BB1368581C10601970C8B210BC70478A
:10BBD800F8B506460F461446D518AC4201D10020E8
:10BBE80007E03A4614F8011B3046FFF7DBFF431C19
:10BBF800F3D1F8BD2DE9F04F9DB00C4617460393DD
:10BC0800064618B183690BB9FFF730FB7C4B9C42A1
:10BC180057D17468A38918075DD52369002B5AD0BA
:10BC28000023099320238DF8293030234FF0010B8E
:10BC38008DF82A30B846454615F8013B002B55D1FA
:10BC4800B8EB070A0BD053463A4621463046FFF771
:10BC5800BFFF013000F0C480099B5344099398F852
:10BC68000030002B00F0BC8000234FF0FF3204931B
:10BC78000793059206938DF853301A930522297875
:10BC88006048FFF7F7FB05F10108049B002831D154
:10BC9800D90644BF20228DF853201A0744BF2B220F
:10BCA8008DF853202A782A2A2CD000210A20079AB6
:10BCB800A84698F800300135303B092B6DD971B38F
:10BCC80026E0514B9C4201D1B468A3E74F4B9C42FC
:10BCD80008BFF4689EE721463046FEF707FB0028B8
:10BCE8009ED04FF0FF301DB0BDE8F08F252BA7D0B8
:10BCF800A846A0E7434A4546801A0BFA00F01843C5
:10BD08000490BBE7039A111D12680391002A01DB16
:10BD1800079204E0524243F002030792049398F812
:10BD280000302E2B10D198F8013008F101012A2B90
:10BD380037D1039B08F102081A1D1B680392002BD8
:10BD4800B8BF4FF0FF330593314D032298F8001028
:10BD58002846FFF78FFB40B14023401B03FA00F051
:10BD6800049B08F101080343049398F80010062285
:10BD7800284808F101078DF82810FFF77BFB0028F9
:10BD880034D0254B03BB039B073323F00703083349
:10BD98000393099B4B4409934CE700FB02320121B2
:10BDA80086E700230A2518460593884698F8002058
:10BDB8000131303A092A03D9002BC5D00590C3E7D1
:10BDC80005FB00200123F0E703AB00932246134B49
:10BDD80004A93046FDF736FDB0F1FF3F8146D8D1C2
:10BDE800A3895B063FF57DAF09987CE703AB009319
:10BDF80022460A4B04A93046FDF7D4FFECE700BF02
:10BE0800D4C0000814C20008F4C00008B4C0000878
:10BE18001AC200081EC200084D980008D9BB0008C5
:10BE280038B50023054C054608462360FCF79EFDFF
:10BE3800431C02D1236803B12B6038BDE0170020F2
:10BE480010B50C46B1F90E1000F0A8F80028ABBFE9
:10BE5800636DA3891B1823F48053ACBF6365A3816A
:10BE680010BD2DE9F0411F468B890546DB050C46C0
:10BE7800164605D502230022B1F90E1000F068F825
:10BE8800A389324623F48053A381B4F90E103B46AC
:10BE98002846BDE8F04100F017B810B50C46B1F9D6
:10BEA8000E1000F055F8431CA38915BF606523F4F4
:10BEB800805343F48053A38118BFA38110BDB1F907
:10BEC8000E1000F013B8000038B5054608461146B4
:10BED8000022054C22601A46FCF7B4F8431C02D134
:10BEE800236803B12B6038BDE017002038B5002364
:10BEF800054C054608462360FCF752FD431C02D159
:10BF0800236803B12B6038BDE017002038B5002343
:10BF1800064C0546084611462360FCF744FD431CC1
:10BF280002D1236803B12B6038BD00BFE0170020A1
:10BF380038B50023054C054608462360FCF738FD54
:10BF4800431C02D1236803B12B6038BDE0170020E1
:10BF580038B50546084611460022054C22601A46A7
:10BF6800FCF728FD431C02D1236803B12B6038BDC0
:10BF7800E017002082B001B901A942B14BB1137892
:10BF88000B601278101C18BF012002B070471046D1
:10BF9800FBE76FF00100F8E77047704738B50546D2
:10BFA800084611460022054C22601A46FCF7D0FCD0
:10BFB800431C02D1236803B12B6038BDE017002071
:10BFC80049B1FF2A8BBF8A230A700360012088BF0A
:10BFD8004FF0FF307047084670470000F8B500BFC3
:10BFE800F8BC08BC9E467047F8B500BFF8BC08BC52
:04BFF8009E467047AA
:10C0000002030405060708090A0B0C0D0E0F101099
:10C0100002030405060708090A0B0C0D0E0F101089
:10C02000457261736572204572726F720D005772AE
:10C03000697465204572726F722025640D0A0000D4
:10C0400000000000000000010203040607080900C8
:10C05000000000010203042530327820005265738D
:10C060006574205374617274200D0000500200202A
:10C07000494E4600696E66004E414E006E616E008C
:10C080003000303132333435363738394142434469
:10C0900045460030313233343536373839616263E2
:10C0A00064656600496E66696E697479004E614E1A
:10C0B0000000000000000000000000000000000080
:10C0C0000000000000000000000000000000000070
:10C0D0000000000000000000000000000000000060
:10C0E0000000000000000000000000000000000050
:10C0F0000000000000000000000000000000000040
:10C10000000000000000000000000000000000002F
:10C1100000000000000000000080E03779C34143C8
:10C12000176E05B5B5B89346F5F93FE9034F384D9D
:10C13000321D30F94877825A3CBF737FDD4F157549
:10C14000000000000000F03F00000000000024405C
:10C1500000000000000059400000000000408F4037
:10C16000000000000088C34000000000006AF840A2
:10C170000000000080842E4100000000D0126341C6
:10C180000000000084D797410000000065CDCD413C
:10C19000000000205FA00242000000E8764837421D
:10C1A000000000A2941A6D42000040E59C30A242BB
:10C1B0000000901EC4BCD64200003426F56B0C4330
:10C1C0000080E03779C3414300A0D88557347643D7
:10C1D00000C84E676DC1AB43003D9160E458E14338
:10C1E000408CB5781DAF154450EFE2D6E41A4B44AD
:10C1F00092D54D06CFF08044F64AE1C7022DB544F2
:10C20000B49DD9794378EA44050000001900000084
:10C210007D000000232D302B2000686C4C006566EB
:10C2200067454647004300504F534958002E0000D1
:10C2300020202020202020202028282828282020D6
:10C2400020202020202020202020202020202020EE
:10C250008810101010101010101010101010101066
:10C260000404040404040404040410101010101046
:10C27000104141414141410101010101010101011F
:10C280000101010101010101010101101010101053
:10C2900010424242424242020202020202020202F0
:10C2A0000202020202020202020202101010102018
:10C2B000000000000000000000000000000000007E
:10C2C000000000000000000000000000000000006E
:10C2D000000000000000000000000000000000005E
:10C2E000000000000000000000000000000000004E
:10C2F000000000000000000000000000000000003E
:10C30000000000000000000000000000000000002D
:10C31000000000000000000000000000000000001D
:10C32000000000000000000000000000000000000D
:08C330004C8EFF7F01000000AC
:04C338000D420008AA
:04C33C00E9410008CB
:10C34000010000001000000000140140000800007F
:10C350000014014000040000001801400400000027
:10C360000014014000080000001401400004000017
:10C3700000180140080000000014014000080000FF
:10C3800000140140000400000018014010000000EB
:10C3900000140140000800000014014000040000E7
:10C3A00000180140200000000014014000080000B7
:10C3B000001401400004000000180140400000008B
:10C3C00000140140000800000014014000040000B7
:10C3D000001001400020000000140140000800008F
:10C3E0000014014000040000001C01401000000087
:10C3F0000014014000080000001401400004000087
:10C40000001C014020000000001401400008000052
:10C410000014014000040000001C01404000000026
:10C420000014014000080000001401400004000056
:10C43000001C0140800000000014014000080000C2
:10C440000014014000040000001C01400001000035
:10C450000014014000080000001401400004000026
:10C46000001C014000020000001401400100000017
:10C470000014014010000000001401400200000000
:10C4800000140140010000000014014040000000C1
:10C4900000140140020000000014014001000000EF
:10C4A00000140140080000000014014002000000D8
:10C4B00000140140010000000020014000200000A5
:10C4C00000140140020000000014014001000000BF
:10C4D00000140140040000000014014002000000AC
:10C4E0000014014001000000001401402000000081
:10C4F000001401400200000000140140000200008E
:10C500000014014000010000001C01400100000077
:10C51000001401400002000000140140000100006E
:10C52000001C014002000000001401400002000055
:10C530000014014000010000000C01400800000050
:10C54000001401400002000000140140000100003E
:10C55000000C01401000000000A24A040008014045
:10C5600000800000001001400008000000100140A1
:10C570008000000000080140008000000010014021
:10C5800000080000001001404000000050020020A0
:10C5900000000000D4C00008F4C00008B4C00008C7
:10C5A000000000000000000000000000000000008B
:10C5B000000000000000000000000000000000007B
:10C5C000000000000000000000000000000000006B
:10C5D000000000000000000000000000000000005B
:10C5E000000000000000000000000000000000004B
:10C5F00043000000000000000000000000000000F8
:10C60000000000000000000000000000000000002A
:10C6100043000000000000000000000000000000D7
:10C62000000000000000000000000000000000000A
:10C6300043000000000000000000000000000000B7
:10C6400000000000000000000000000000000000EA
:10C650004300000000000000000000000000000097
:10C6600000000000000000000000000000000000CA
:10C670004300000000000000000000000000000077
:10C6800000000000000000000000000000000000AA
:10C690004300000000000000000000000000000057
:10C6A000000000000000000000000000000000008A
:10C6B0004300000000000000000000000000000037
:10C6C000000000000000000000000000000000006A
:10C6D000C9BF00087DBF0008000000002FC200088D
:10C6E0002DC200083EC000083EC000083EC0000841
:10C6F0003EC000083EC000083EC000083EC0000822
:10C700003EC000083EC00008FFFFFFFFFFFFFFFF25
:10C71000FFFFFFFFFFFF00000100415343494900B5
:10C720000000000000000000000000000000000009
:10C730000000000000000000000041534349490090
:10C7400000000000000000000000000000000000E9
:0CC75000000000000000000000000000DD
:0400000508009665F4
:00000001FF
